:020000040800F2
:103000000080002077B70008F1B40008F3B400088E
:1030100000000000000000000000000000000000B0
:10302000000000000000000000000000F5B40008EF
:103030000000000000000000F7B400084D88000800
:1030400095B3000897B3000899B300089BB3000834
:103050009DB300089FB30008A1B30008A3B3000804
:10306000A5B300085D880008A7B30008A9B300084D
:103070004D890008ABB30008ADB30008AFB300083A
:10308000B1B30008B3B30008B5B30008B7B3000884
:10309000B9B30008BBB30008BDB30008BFB3000854
:1030A000C1B30008C3B30008C5B30008CFB7000818
:1030B000C7B30008D7B70008C9B30008CBB30008EE
:1030C00001000000000000000A00000000000000F5
:1030D0006400000000000000E803000000000000A1
:1030E0001027000000000000A08601000000000082
:1030F00040420F0000000000809698000000000091
:1031000000E1F5050000000000CA9A3B0000000045
:1031100000E40B540200000000E8764817000000AD
:103120000010A5D4E800000000A0724E18090000AD
:1031300000407A10F35A00000080C6A47E8D030080
:103140000000C16FF286230000008A5D78456301AC
:10315000000064A7B3B6E00D0000E8890423C78A25
:10316000034C206804348047FBE701F0BFFFFEE713
:0431700034C500085A
:10317400014802490160704708ED00E00030000892
:10318400B0B51E4D2C1F20688006400F411E032938
:1031940022D81B487944097949008F442301171A1E
:1031A400296803220A40032A00D0164829684906E0
:1031B400490F491C06F0F6FE29684904490E4843A4
:1031C4002968490F491C06F0EDFE0BE07D20000242
:1031D40008E00120C00305E00C3D28688004410F8D
:1031E4000848C84008490860226892093C231340F3
:1031F400064AD258D0400860B0BDC0460C10024008
:1032040000127A000024F4005C0B0020E0B10008F6
:1032140010B5816A8B6D8A6D5024234205D0D20685
:1032240002D4096D496B884710BD012043021A433B
:103234008A650A68D3681B059B0F02D0104908678A
:1032440010BD8B7E002BF9D113681B07F6D593684C
:103254005B0709D4583153680C24A3435360FF23FC
:1032640002330A689A4305E08A6D202313438B6571
:10327400CA6D5C3102430A600149086710BDC0464B
:04328400E809002035
:10328800F0B587B005460020049006900124E602B8
:10329800E94A1068E949884206D03246AC32E84823
:1032A800E84906F0D7FFE44A2868E74988420DDC78
:1032B800F449884218DDF44988422ADCF6498842F4
:1032C80042D0F64988423FD0F5493BE0DF49884281
:1032D80014DDDF49884224DCE149884234D0E149E1
:1032E800884231D0E0492DE0EE49884221DDEE499F
:1032F800884229D0012827D0EC4923E0DB498842BD
:103308001CDDDB4988421FD0DA4988421CD0DA49E3
:1033180018E0DE49884217D0DD49884214D0DD49DB
:1033280010E0CC4988420FD0CB4988420CD0CB4919
:1033380008E0DF49884207D0DE4903E0CF498842E8
:1033480002D0CF49884269D10595A868002809D0DC
:10335800D949884206D03246AE32B948B94906F052
:1033680079FFB54A3546106904263043D34FB84231
:1033780007D105984068401E02281AD32A46B3325E
:1033880012E0D069401E082806D32A46B732AC4856
:10339800AC4906F05FFFA84A059840680221C84179
:1033A800082806D32A46B932A548A64906F052FF8E
:1033B800A14A5423D05C012802D1022007B0F0BDF5
:1033C800D45410688168490717D41169059A52685E
:1033D800022A17D104221143B9422BD1B849C94353
:1033E800059A1268D3430B43816A194054238162BA
:1033F8000024002A23D4904AAAE0906D202101439A
:103408009165A5E003933143B942AD4F24D1059CA2
:1034180021680F40826A3A4382628BE03246AD32BD
:103428008748884906F016FF834A0595A86800284A
:103438008ED197E7059802680024002ADBD5A248B8
:103448000168994B9A424FD09A4B9A424FD0984B69
:103458009A4255D1052248E01F2313400F240194B6
:103468009C407549096EA143029105990968394242
:1034780037D0CF07049F4BD18F0744D44F0744D48C
:103488000F0744D4CF06374642D48E0600D5BAE09B
:103498004E0600D5B9E00E0600D5B8E0CE0500D539
:1034A800B7E08E0500D5B6E04E0500D5B5E0294257
:1034B80000D0B4E0CE0400D5B3E08E0400D5B2E06D
:1034C8004E0400D5B1E00E04019F21D4CE0300D5EF
:1034D800ADE08E0300D5ACE04E03F6171227374057
:1034E80016E04E00F70E13E00322920501E00322D6
:1034F800D2051140072292050368934359180160C9
:103508004D4A542324E0012702E0022700E0032764
:103518009F40029D2F43484E37669208F6699642AF
:1035280007D9E243846A14408A00120F9A40224362
:103538008262059C0A0243699343A4681440614A65
:1035480022401A4342610024002906D43A4A039BC8
:103558000498D054204607B0F0BD01265A480068A8
:103568000722930502461A40514FB94230D1F70558
:1035780005463D402CD154490868984302433A43D4
:103588000A6052480068524906F00AFD0C2141437E
:10359800481C069006980028D8D0274A039B06980E
:1035A800401E069006980028D2D00698401E069025
:1035B80006980028CCD00698401E06900698002849
:1035C800C6D00698401E069006980028E7D1BFE7A7
:1035D800354DA9420AD1370605463D4006D13A493C
:1035E8000868984302433A430A60AFE7314DA9425D
:1035F800ACD1B1050840A9D1334D2868984302439E
:103608000A432A60A2E7052782E7062780E70727FB
:103618007EE708277CE709277AE70A2778E70B2758
:1036280076E70C2774E70D2772E70E2770E7102757
:103638006EE711276CE7C046640A002000240140A9
:1036480071C0000814BE0008FF000020FF1F0034EE
:10365800FFFF004000000140000002440000044851
:1036680000200034004000380080003CFF030028A0
:10367800000400280008002C001000300001002081
:1036880000020024030000081F000014200000149A
:10369800400000188000001C040000080800000C0E
:1036A80010000010FF3F00B8004000B802000004FE
:1036B800001000B0002000B404FFFF0704000080E1
:1036C800FFFF070000FFFF07082701405C0B0020F1
:0436D800400D03009E
:1036DC00F0B58DB00446002306930120002C00D1D8
:1036EC00D2E121680A68002A00D5CDE103930427B2
:1036FC003943FF250235404EB14203D120690028E1
:10370C0008D113E03D483E492A4606F0A1FD206948
:10371C0000280BD001210A02904207D049028842AE
:10372C0004D06A1C3548364906F092FD6069F841B0
:10373C00092804D3AA1CD648D64906F089FD0127CE
:10374C00F803E1690143814204D0EA1CD048D14915
:10375C0006F07EFDB904E06808430191884204D06C
:10376C002A1DCB48CB4906F073FDA0691021C84136
:10377C00042804D36A1DC648C64906F069FD206AB0
:10378C00C549884208DC002814D03905884211D07C
:10379C00790588420ED008E0B90588420AD0F905AF
:1037AC00884207D03906884204D0AA1DB848B949C6
:1037BC0006F04EFD606A322800D96DE0784400793D
:1037CC00400087441F696969696969696969696940
:1037DC0069696969691F1F696969696969696969E1
:1037EC0069696969691F1F696969696969696969D1
:1037FC0069696969691F1F000402014071C00008F2
:10380C009ABA0008606800280DD0F90288420AD0E4
:10381C000321C902884206D02A4608329C489D4999
:10382C0006F016FD606822462832002812D0A068E7
:10383C0002280FD3B90388420CD005210903884212
:10384C0008D00B359248934916462A4606F000FDDF
:10385C0032468E4E0492507800284FD10025E562F6
:10386C0015700C950B950A95099508950520000780
:10387C002168B14219D0894A91423FD188490A68DE
:10388C003A430A6009683940079102210891079967
:10389C00F902059102901EE0EA1D7D487D4906F073
:1038AC00D7FC60680028B0D1BDE77D490A683A436F
:1038BC000A600A683A400792079A0A6802231A4378
:1038CC000A600968194007910C21089107997549FC
:1038DC000291202105910A950321099108AE3146E8
:1038EC0000F0E6FA07200C900B950A95022009903F
:1038FC00059808900298314600F0DAFA0597256889
:10390C00286802902A686849114026460C364CCE2D
:10391C001E43A369E769206A3043184338431043B8
:10392C000843286061680320C00281425B4E09D0C5
:10393C000598C20291420DD1306890433060716895
:10394C0011430DE00598C002316801433160716884
:10395C00814305E03068554A104030607168114071
:10396C00039F7160A16801290DD0052000038142DD
:10397C000ED005988203914212D13068104330600A
:10398C007168914312E0059880033168014303E0AC
:10399C00059880033168814331607168014305E00B
:1039AC003068434A1040306071681140716028687B
:1039BC008006800F26D030200299014022D13D484C
:1039CC0000683D4906F0EAFA142141430691069835
:1039DC00002817D00698401E06900698002811D093
:1039EC000698401E0690069800280BD00698401E9C
:1039FC0006900698002805D00698401E069006985A
:103A0C000028E7D1B5420FD0019D616A8A072B4887
:103A1C0010D0CB062A4B11D41C68AC431C608C060E
:103A2C0011D55C682C4310E005984504616A8A073F
:103A3C002248EED10168A943016019E01C682C43AF
:103A4C001C608C06EDD45C68AC435C60DD601D6171
:103A5C00002A08D40268AA430260C90708D0011FD3
:103A6C000968294307E002682A430260C907F6D1B6
:103A7C00011F0968A943049A001F016050780028AF
:103A8C0001D10598507038460DB0F0BD04020140CC
:103A9C0071C000089ABA0008FFFF3F000002014005
:103AAC0034100240000400500F7400FEFFF7FFFFBB
:103ABC00FFBFFFFF5C0B0020400D03008418024089
:043ACC00001802409C
:103AD00070B582B00026019600280DD0054600681A
:103AE0000168002908D4042108432149884206D1ED
:103AF0002920285C01280BD0012002B070BD1D4890
:103B00001D491E4A06F0AAFB2920285C0128F3D192
:103B100028682935016801220A43026002202870C2
:103B200017480068174906F03FFAC0000190019855
:103B300000281AD00198401E01900198002811D049
:103B40000198401E0190019800280BD00198401E5A
:103B500001900198002805D00198401E019001981D
:103B60000028E7D1304602B070BD02B070BDC0463B
:103B70000402014071C000089ABA00081F03000047
:083B80005C0B0020400D030066
:103B8800F0B585B0574C2178002902D0022005B045
:103B9800F0BD02900393012727707D20C100606A61
:103BA800049141183E04504D2868304216D0636A8B
:103BB80003208B421AD22B6833420FD0636A8B42A0
:103BC80014D22B68334209D0636A8B420ED22B6819
:103BD800334203D0636A8B42E6D307E0286843493F
:103BE8004B1C01932B600842384603D000212170FA
:103BF80005B0F0BD606A049941180120009087045F
:103C08002868384216D0636A03208B42EED22B68AC
:103C18003B420FD0636A8B42E8D22B683B4209D003
:103C2800636A8B42E2D22B683B4203D0636A8B42C1
:103C3800E6D3DBE7686800990843686002990A6080
:103C4800BFF36F8F03984860606A04994118286829
:103C5800304216D0626A03208A4219D22A68324258
:103C68000FD0626A8A4213D22A68324209D0626A45
:103C78008A420DD22A68324203D0626A8A42E6D367
:103C880006E028680199296018490842009807D079
:103C98006968009A914369600021217005B0F0BD00
:103CA800606A049941182A6800203A42F0D0636A91
:103CB80003228B4213D22B683B42E9D0636A8B42C2
:103CC8000DD22B683B42E3D0636A8B4207D22B6844
:103CD8003B42DDD0606A88421046E4D3D8E703202F
:103CE800D6E7C046E809002010200240FAC30000C9
:103CF800F0B587B00446684D287C002804D1674891
:103D08006749A02206F0A6FA2878002802D00220E7
:103D180007B0F0BD0594012129707D20C200686AB2
:103D2800069282180C045F4E3068204219D06B6AE4
:103D38000320934211D23368234212D06B6A934214
:103D48000BD2336823420CD06B6A934205D2336896
:103D5800234206D06B6A9342E6D30021297007B04C
:103D6800F0BD3068504B5A1C049232601842084625
:103D7800F3D1686A069941180120039087043068D6
:103D8800384216D06A6A03208A42E6D232683A423A
:103D98000FD06A6A8A42E0D232683A4209D06A6A27
:103DA8008A42DAD232683A4203D06A6A8A42E6D351
:103DB800D3E70022D04305990860287DA96C08182C
:103DC80081425AD201924029029106D3334834499C
:103DD800364A06F03FFA0299334B7068344A10406D
:103DE800C9000143A01C08437060686A069941181D
:103DF8003068204216D06A6A03208A4240D232686C
:103E080022420FD06A6A8A423AD23268224209D0E4
:103E18006A6A8A4234D23268224203D06A6A8A4283
:103E2800E6D32DE0306804993160184227D1686ADA
:103E3800069941183068384216D06A6A03208A42C7
:103E48001ED232683A420FD06A6A8A4218D2326861
:103E58003A4209D06A6A8A4212D232683A4203D098
:103E68006A6A8A42E6D30BE0287DA96C0818029991
:103E7800491C8142A7D3019805E0002003E003987C
:103E88000599029A0A6071680222914371600021C3
:103E9800297007B0F0BDC046E809002071C00008CD
:103EA80004BB000810200240FAC3000052020000C0
:043EB80005FEFEFF06
:103EBC00F0B58DB00B4604460B20000721180A20E4
:103ECC00C141039104290C9307D3052905D09848C7
:103EDC009849B12206F0BCF90C9B1868010C02D170
:103EEC0080B2002805D192489249B22206F0B0F96E
:103EFC000C9B58689049884207941CDC122800D906
:103F0C000BE1012181408D48014200D105E1986807
:103F1C00032805D386488749B42206F099F90C9BEF
:103F2C001A68002A00D1EAE0012005908B488442EF
:103F3C000FD005200EE08249884200DDE1E0844983
:103F4C008842E4D083498842E1D083498842DED05C
:103F5C00E3E003200190059D2804029000270B97B5
:103F6C003C46099711E021437160089C1A68104681
:103F7C00E840BF1C0B99091D0B9108346D1C099965
:103F8C00491C0991002800D1B9E0681E059E0A90D1
:103F9C0086403240EAD0586812280492089423D8FC
:103FAC0001218140704A11421ED0D868042806D3E2
:103FBC00C4225F485F4906F04BF90C9BD868B840A7
:103FCC000321B940079CA2688A430243A260586847
:103FDC00C206D20F0A9B9A406368B34313436360D3
:103FEC000C9BCA433E4605E00321B940CA430999DC
:103FFC004E00079CE168069211409A68B2400A4351
:10400C00E2601021014312291DD10398042841D2EA
:10401C001869082806D3DD224548464906F018F9E8
:10402C000C9800691C210B9A11400F228A400A9BA4
:10403C00DB089B00E3181C6A944388402043079CD0
:10404C0018620C984068226806990A4003210346BE
:10405C000B40B340134323600C9BC000089C85D5D8
:10406C00182020400F2383400A9A8A433C4EB118F3
:10407C000A6E9A43603105231B07079C9C4212D0A1
:10408C003A4B9C4211D03A4B9C42019B049C0ED162
:10409C0002230CE00528BBD0DC222548254906F07C
:1040AC00D7F80C9BB4E7002300E00123049C834069
:1040BC0013430B602B4801680C9B5868029A104202
:1040CC0001D0214300E0A143264A116051688203CC
:1040DC0001D5214300E0A143224A51603168C2025C
:1040EC0005D5214331607168800206D53BE7A143B9
:1040FC0031607168800200D535E7A14334E70DB01B
:10410C00F0BD1049884200D101E70F49884200D127
:10411C00FDE60E49884200D1F9E605480549B3226F
:10412C0006F096F80C9B9868032800D3F2E6F7E6A5
:10413C0071C0000872BB0008FFFF10100F000600D2
:10414C00FFFF21100000221000003110000032107F
:10415C00000011100000121000002110000C005083
:10416C0000180240801802400600060000040050AF
:04417C0000080050E7
:10418000F0B581B00446744B00280CD0201F0221EA
:10419000C84103280CD88000704908581946042CDF
:1041A0000BD175310AE01946743118466E3005E0BE
:1041B000184673301946042CF3D077310778186B02
:1041C0000D780126B107009188420BD064498842DE
:1041D00008D0644988420BD102212246CA41062AEE
:1041E0000FD21EE002212246CA41042A09D218E059
:1041F000002C02D15C49884213D05C49884200D12E
:10420000A4E05B494118B002814348424841002C78
:1042100001D1002805D157485749584A06F01EF8E1
:104220004D4B012F00D083E0012D00D080E0002C09
:104230000FD0211F0220C14103291DD879440979DB
:1042400049008F44011E23296F215854042C21D189
:1042500026E06E2002211954742019541D6B484A1F
:10426000954223DC0098854238D03D48854235D0C0
:104270003D48854232D029E073215854042C09D19D
:104280000EE070215854042C04D109E071215854D7
:10429000042C05D0772104E072215854042CF9D164
:1042A000752158541D6B364A9542DBDD35488542F1
:1042B00006DC2C48854211D02C4885420ED005E002
:1042C000314885420AD03148854207D029482A49D9
:1042D0002F4A1F4605F0C2FF294A3B4602212046CD
:1042E000C841062826D21F2004403046A040296A33
:1042F00081432962296A01432962186B904206DCD6
:104300000099884209D01649884206D00DE0174925
:10431000884202D01349884207D182681D49114062
:10432000062905D03204914202D001683143016070
:1043300001B0F0BD0F28D6D01548421C0D480E49DB
:104340001F4605F08BFF0E4A3B46CCE70421214374
:10435000042900D165E754E76C09002090B20008F9
:1043600000040040002C01400020004000400140BB
:1043700000BCFEBF71C000084FBF00082408000049
:10438000FF2B0140FF430140004401400048014031
:08439000F41D0000070001000C
:10439800F0B583B00E4604468548006B854D8649C6
:1043A800884209DD8549884211DC8749884219D04D
:1043B8008649884216D010E001218907884211D029
:1043C800834988420ED0834988420BD005E07C4956
:1043D800884207D07B49884204D07F487F492A46D3
:1043E80005F038FF20680A2840D8012181407C4820
:1043F80001423BD06068401E032804D3AA1C7648BB
:10440800764905F027FFA0680227F841042804D35D
:10441800EA1C7148714905F01DFFE068102804D3B3
:104428002A1D6D486D4905F015FF6C226049885CAE
:10443800012800D1B9E001278F54042E02921FD021
:10444800002E28D1096B086AB84308625A4881428D
:104458008D69E0680190226860680B6A4FDCBE07CE
:10446800B14252D05A4EB1424FD083E06A1C5A48EA
:104478005A4905F0EFFE6068401E0328BED2C2E725
:10448800086B4D49884244DCB90788424FD05049EF
:1044980088424CD043E0086BB90788420DD04C499C
:1044A80088420AD04849884207D03A354A484B4999
:1044B8002A4605F0CFFE3E48006B3903026A8A435C
:1044C800026261680902474A0A40E168090389B241
:1044D8008918F3221202C36993430B43016AC3612B
:1044E8000522520323681B0313409143C918016234
:1044F80003218902C2698A43C2611C3037E0334E06
:10450800B14202D0304EB14234D10326B5430543FF
:1045180031E02D4988420AD02C49884207D01A3503
:104528002D482E492A4605F095FE2148006B016A60
:10453800102291430162616809022A4A0A40E1682F
:10454800090389B28918F3221202836993430B4342
:10455800016A836122681201A0231A4099438918CD
:1045680001620321890282698A4382611830A16845
:10457800090213E03D4308461830F026B543019E72
:104588003601F6B2AD198D610A252A40AB439A1857
:104598000A628A690C239A438A61A1680027044A3F
:1045A800029BD75402680A430260384603B0F0BD44
:1045B8006C090020EA0F0000FF2B0140FF43014077
:1045C8000044014000480140002C014000400140E7
:1045D800000400400020004071C000084FBF0008E0
:0845E80005040000000FFFFFB5
:1045F000F0B583B09748401C974F79688142974E39
:1046000004D397489749324605F028FEB868002839
:104610000BD001210A03904207D00907884204D039
:10462000721C8F488F4905F019FEF86839688E4C66
:10463000A14212D00C21C841042805D332460832C9
:104640008748884905F00AFE0120C002396A014303
:1046500081420CD03246093205E00121490308436A
:10466000884204D0321D7E487E4905F0F7FD386946
:1046700000280DD001218902884209D00321490276
:10468000884205D032460C327548764905F0E6FD81
:1046900078690C25002801D0A84305D032460D3298
:1046A0006F48704905F0DAFD0195B8690821C841E5
:1046B000042805D332460E3269486A4905F0CEFD1A
:1046C00001200290C503F8692843A8424FD1786AB7
:1046D0000C2805D31036F048F049324605F0BEFDEF
:1046E0003E683168EF480840B9683A690A437B6917
:1046F0001343F9690B437A6E1A4302433260032075
:104700000090000372688243F868104370600022D2
:10471000A642104600D0386ABB690343B068E24C39
:1047200004401C43B460F06A0F2398433C467B6A04
:104730001843F062DD4886420DDDDD488642D84FE1
:1047400026D0BE421DD0DB4886420BD1DC48C06C6F
:104750008007000F1AE0D84886425FD0D7488642CB
:10476000CF4F15D01022D848BE4214D160E0324657
:104770000F32C948C94905F071FD786A0C28A9D2E1
:10478000AEE7CF48C06C000A019A1040CD4A1258DB
:10479000CD48BE424CD0A94220D1082A00D974E0AD
:1047A000274652007A4492885200974408006301D9
:1047B000360163017C006301630163018800C34823
:1047C0000068BF490968890A1C220A40C049895803
:1047D0001F220A40D04000D01FE14AE1082A54D8E5
:1047E000274652007A4492885200974408004301B9
:1047F000330143016A004301430143017600B3489A
:104800000068AF490968890A1C220A40B0498958E2
:104810001F220A40D04000D01CE12AE1A848C06C09
:10482000019A1040A74A12589D4FA748BE42B2D1E4
:10483000082A2AD8274652007A4492885200974480
:1048400015001901C60019012600190119011901E5
:10485000C400C04600127A00DC080020150C0000DD
:1048600071C00008DCBB0008008000409748006869
:1048700093490968890A1C220A40954989581F22D0
:104880000A40D04000D0A2E0F3E02746F2E08C4C92
:1048900021688906490F22D0226838210A40082A57
:1048A00023D17C4893E0864C21688906490F3CD08F
:1048B000226838210A40082A43D17648ADE02846CC
:1048C000ABE07F4C21688906490F34D0226838213B
:1048D0000A40082A55D16F48BCE02846BAE0083C97
:1048E00021688904490FC84071E022680A40102AF3
:1048F00067D11D466168009A11400329654A00D0BE
:10490000024660684006400F411C104605F04CFB13
:1049100061684904490E48436168490F491C05F024
:1049200043FB2B46002852D1A3E0083C21688904B0
:10493000490FC84071E0083C21688904490FC8400C
:1049400088E022680A40102A5CD11D466168009AFE
:10495000114003294F4A00D0024660684006400FCC
:10496000411C104605F020FB61684904490E48438C
:104970006168490F491C05F017FB2B4600284CD1F4
:1049800077E022680A40102A59D11D466168009AD2
:10499000114003293F4A00D0024660684006400F9C
:1049A000411C104605F000FB61684904490E48436C
:1049B0006168490F491C05F0F7FA2B46002849D1D8
:1049C00057E02068084020285CD10120C00359002E
:1049D000404A515A05F0E8FA7A68009951438842F2
:1049E00048D31103884245D8010E54080002002321
:1049F0000019594105F0FCFA38494118384A9142EA
:104A000035D337E0206808402028284605D02068A4
:104A1000084018282CD17D20000259002D4A515AF7
:104A200005F0C2FA400079684A08101805F0BCFA8F
:104A3000294901401ED00007400F084317E02068B5
:104A400008402028284605D02068084018280FD1A3
:104A50007D20000259001F4A515A05F0A5FA7968D5
:104A60004A08101805F0A0FA80B2102802D3F060AE
:104A7000002002900020386778671A48B8660298CC
:104A800003B0F0BD206808401828F1D17D20000255
:104A90009DE7C04600127A0071C00008DCBB000828
:104AA00000800040F369FFCFFFF4FF11FF4B00408F
:104AB000004C0040003801400044004000480040E5
:104AC0000810024040B200080024F4005C0B0020F3
:104AD00020B2000812B90008F0FF000000FDFFFF3F
:084AE00000FD0F0001000100C0
:104AE80070B5774DA86A010A764C0FD1C10715D168
:104AF800810728D441073CD4010750D4C10664D4A7
:104B0800810678D4400600D58BE0C0E06E486F4936
:104B1800224605F09FFBA86AC107E9D001214E048F
:104B2800E96A0A463243B24206D0621D66486749BE
:104B380005F090FBA86AE96A2A685368B3430B43F7
:104B480053608107D6D501210E04296B0A463243EA
:104B5800B24207D022460C325B485C4905F07AFB2A
:104B6800A86A296B2A685368B3430B43536041070B
:104B7800C2D501218E04696B0A463243B24207D07E
:104B8800224613325048514905F064FBA86A696B04
:104B98002A685368B3430B4353600107AED501211C
:104BA800CE03A96B0A463243B24207D022461A32D4
:104BB8004548464905F04EFBA86AA96B2A68536820
:104BC800B3430B435360C1069AD501210E03E96B29
:104BD8000A463243B24207D0224621323A483B497C
:104BE80005F038FBA86AE96B2A689368B3430B435E
:104BF8009360810686D501214E03296C0A4632430B
:104C0800B24207D0224628322F48304905F022FB0D
:104C1800A86A296C2A689368B3430B4393604006DB
:104C280035D528682A49884208D02A49884205D0BB
:104C380022462F322448254905F00CFB01200605A1
:104C4800696C08463043B04206D0224630321E48CE
:104C58001E4905F0FFFA696C28684268B2430A43A6
:104C68004260B14213D1A96C15220B46D341042BE3
:104C780007D3224635321448144905F0EBFAA96CDB
:104C8800286803225205436893430B434360282056
:104C9800285C000612D50120C604E86C01463143A1
:104CA800B14206D03D3408480849224605F0D2FAF8
:104CB800E86C29684A68B24302434A6070BDC0463E
:104CC800DC080020E10C000071C00008DCBB000813
:084CD8000044004000380140D7
:104CE000F0B581B08C20364900220A50354B5C6A01
:104CF00008680168090716D5C169890213D4012122
:104D00004F050091CE02304D02E0C16939420AD10F
:104D1000596A091BA94201683DD84907F5D5C169FF
:104D20003142F2D018E00168490728D5C16949022B
:104D300025D401218F050091CE02234D02E0C169E7
:104D400039421CD1596A091BA942016823D8490775
:104D5000F5D5C1693142F2D006620D2149010368DF
:104D60008B4303608168009B9943816084202021EC
:104D7000134C215020468C302346883318E0842081
:104D800020210F4C215088202150E26610468021BE
:104D9000625401B0F0BD0D235B019943016081684D
:104DA000009B99438160064C20468830234684331B
:104DB00020211960016003208021625401B0F0BD00
:0C4DC000DC080020E8090020FFFFFF01D4
:104DCC0070B58421415821291AD102465632938A52
:104DDC00002B15D00168104C02E05B1E1D040FD097
:104DEC001588002D0DD0CD692D06F6D5056D2E88B4
:104DFC0026408E62AD1C056515886D1E1580ECE78E
:104E0C0070BD0120C0058A6882438A600868402210
:0C4E1C0002430A6070BDC046FF010000A8
:104E280010B58421415821290FD1014656310A88ED
:104E3800002A0BD0026D1388094C1C4003689C6241
:104E4800921C02650888401E088010BD0068016831
:104E5800802291430160016840220A43026010BD2C
:044E6800FF01000046
:104E6C00F0B586B00168CA690F688E688823C3588C
:104E7C00222B79D105465E3520246B89002B0094BA
:104E8C0075D0224073D03246064688366B88039321
:104E9C0001231A40049205931A0217400197876D5B
:104EAC00029502E0C266A20661D5496A039A1140D6
:104EBC0039702988491E2980816D4F1C87650168CE
:104ECC00CC6962072AD0019B5D425D41E307059BDB
:104EDC0000D02B46002B04D101230B6275681D43B7
:104EEC007560049B5D425D41A307059B00D52B4675
:104EFC00002B05D102230B62736804251D437560DA
:104F0C00049B5D425D41002A059A20D4002A20D0E2
:104F1C007268002A029D01D0002272602A88002A41
:104F2C00C1D1012212020B6893430B608A68194BA2
:104F3C001A408A602022326000220267C36E012B65
:104F4C00B0D10B681025AB43029D0B60AAE72A0079
:104F5C00DED104220A627268022313437360726802
:104F6C00002A029DD8D1D9E7183108220DE02A88F1
:104F7C00002A0DD06B899A420AD2074A026705486B
:104F8C00401C8A6802408A60009A086810430860D6
:0C4F9C0006B0F0BDFEFFFFEF21B40008DE
:104FA800F0B586B004460168CA690B688D68882028
:104FB800205822287BD10495019325465E35202070
:104FC80000906889002875D00098024072D0264663
:104FD800883668880390012204981040049005924E
:104FE80010021A4602400192A76D029402E0E2669E
:104FF80098065FD5486A039A104038802888401E72
:105008002880BF1CA765CB695A072AD0019844425B
:105018004441D807059800D02046002804D1012033
:1050280008627468044374600498444244419807D1
:10503800059800D52046002805D10220086270682E
:10504800042404437460049844424441002A0598A7
:1050580020D4002820D070680028029C01D00020AD
:10506800706028880028C3D1012000020A688243A2
:105078000A608868194A1040886020203060002241
:105088002267E06E0128B2D108681024A043029C70
:105098000860ACE72000DED10420086270680222B4
:1050A8000243726070680028029CD8D1D9E7183191
:1050B80008220DE0288800280DD06A8990420AD27B
:1050C800074820670548401C8A6802408A60009AA1
:1050D80008681043086006B0F0BDC046FEFFFFEF49
:0450E8008BB400087D
:1050EC0000B5C7B0AD4A1068FF21359160313791DA
:1050FC005F393291084310607D203890C400A84E6F
:10510C003068214604F04AFF401E010E0127002999
:10511C0028D1A4494860A44A1368A44E3340032004
:10512C0085075B19136000238B6007230B601168E4
:10513C0031409B4E11609E490F719E4BD96839438B
:10514C00D960D96839404291429939079A680A4323
:10515C009A609A680A4042924299400296490A68BB
:10516C0002430A6003203A904202944D28461438B8
:10517C0001683092914301223B9252023492891879
:10518C00016031682868319426461836304229D09F
:10519C00062048438A4904F001FF0221081A03281B
:1051AC0020D0821E514251412A6832423A4600D0E8
:1051BC000A46002A16D1421E514251412A683242F7
:1051CC003A4600D00A46002A0CD1414241412A6895
:1051DC0032423A4600D00A46002A03D1001D296803
:1051EC003142DCD13397734C27462C3F3968254626
:1051FC00283D28683A9A8243382039900140102380
:10520C000846369358408018434243413B98420429
:10521C00204634380829016825D0002B23D13B9B2C
:10522C001B041943016062494B6A046814421AD189
:10523C004C6AE41A642C14D80468144213D14C6AD6
:10524C00E41A642C0DD8046814420CD14C6AE41A8C
:10525C00642C06D80468144205D14C6AE41A652CF7
:10526C00E3D372B6FEE72E964C49096807212F91BD
:10527C0009033B680B433B603B68524C23403B604B
:10528C0003681342399C01D172B6FEE73A683B9B26
:10529C001A4306232D939A433A60454A526A3B6857
:1052AC002340082B21D0424B5B6A9B1A464EB342DB
:1052BC00EAD83B682340082B17D03D4B5B6A9B1AFE
:1052CC00B342E1D83B682340082B0ED0384B5B6AC5
:1052DC009B1AB342D8D83B682340082B05D0344BDB
:1052EC005B6A9B1AB342DAD9CEE72C4A1268520792
:1052FC002CD02A4E32682F9B9A4332602C4A526A29
:10530C00264B1B685B0721D0294B5B6A9B1A2E4EE0
:10531C00B342B9D8214B1B685B0717D0244B5B6A8F
:10532C009B1AB342B0D81D4B1B685B070ED0204BA9
:10533C005B6A9B1AB342A7D8184B1B685B0705D056
:10534C001B4B5B6A9B1AB342DAD99DE73A688A43D6
:10535C003A6039688906490F3CD0386820400828E3
:10536C001A483CD039682140102900D03FE1296807
:10537C003A9A11400329389C00D0154829684906EF
:10538C00490F491C04F00AFE29684904490E484398
:10539C002968490F491C04F001FE21E0002002405D
:1053AC005C0B002010E000E020ED00E0FFFFFF00B0
:1053BC00E809002034100240000001401470004045
:1053CC0040420F00FFF0FFFF8813000000127A002C
:1053DC000024F40000688004410FCB48C840389C7E
:1053EC00396889093C252940C84A51581F2739403A
:1053FC00C840C7490860E10004F0D0FD401EC54913
:10540C00884200D940E7C4490979C44A5060C44C69
:10541C002068C04B18403A9B9B07C01820600026A0
:10542C0096602F981060002900D12DE720972068F6
:10543C00B849084020603398B74908712B95B94C8E
:10544C00206A3A9A90432062206A23939843206200
:10545C003B9DA805216A81432162469645962068AA
:10546C0004212C9108432060206808403D903D9811
:10547C0020682021389108432060206808403D9026
:10548C003D98206828432060206828403D903D9836
:10549C0020680221084320602068259108403D9037
:1054AC003D98206808212A91084320602068084014
:1054BC003D903D989C480F2129910161449643925F
:1054CC0014469A4842909A481838289042AF394668
:1054DC00FEF7EEFC449643942C984290954839463E
:1054EC00FEF7E6FC44964394E8031C90401C429063
:1054FC0005201F90000721903946FEF7D9FC4496F1
:10550C00439428041E90223842908B4C20463946F6
:10551C00FEF7CEFC449543962A9842902046394695
:10552C00FEF7C6FC459644964395299842907E48D2
:10553C0018383946FEF7BCFC40207D49086144967A
:10554C0043951D90429028983946FEF7B1FC754959
:10555C0048682843486048682840429042983598EB
:10556C000002764A116881431160754934980860CD
:10557C00744A2B9815542C20289015546F070C2026
:10558C002290106456649664D76416632F98506307
:10559C00906356629662101D06772C98D0619576B2
:1055AC00168369052C056848199051C2166027911D
:1055BC0051602A9890603F963E963D9626960C3AFE
:1055CC003C96D068389908432028379D06D02A4647
:1055DC0036325E485E4904F03BFE5A4A1069002898
:1055EC000CD50121C907884214D05A4909E0386802
:1055FC00204020283BD13B98C003F0E60AD03B99D1
:10560C004905884206D02A4637325048504904F0A2
:10561C001FFE4C4A907E022806D32A4638324B484D
:10562C004B4904F015FE474A906A0A211B91C84168
:10563C00042806D32A4639324448454904F008FE6A
:10564C00404A506A4449884207DC4449884215DC88
:10565C00002823D0012189021DE04149884214DC35
:10566C0013218901884219D01F99090213E0386867
:10567C002040182800D181E10020B0E611218901D9
:10568C0088420BD00921C90105E015218901884206
:10569C0004D017218901884200D072E12898105C4F
:1056AC00022806D32A463B322848294904F0D0FD6B
:1056BC00244A5069042808D0082806D02A463C32CF
:1056CC002248234904F0C4FD1E4A3B980103106B89
:1056DC0008431A91884245D1107E02284CD2507E44
:1056EC00022853D2506B08285AD2906B082861D2EA
:1056FC002B98105C022868D2D06C3843B8426FD11A
:10570C001069002876D18FE00024F400E0B1000885
:10571C005C0B0020FFFFFF00E809002010E000E018
:10572C0020ED00E034100240180C0050C0E00000E6
:10573C0018080050001400500004005008E400E069
:10574C0000E100E0640A00200024014071C0000860
:10575C0014BE000804000080BF0400003F040000D9
:10576C003F0500002A463D32FB48FC4904F070FD21
:10577C00FB4A107E0228B2D32A463E32F648F7493D
:10578C0004F066FDF64A507E0228ABD32A463F321F
:10579C00F148F24904F05CFDF14A506B0828A4D39F
:1057AC002A464032EC48ED4904F052FDEC4A906B2D
:1057BC0008289DD32A464132E748E84904F048FDC1
:1057CC00E74A2B98105C022896D32A464232E248CC
:1057DC00E24904F03DFDE24AD06C3843B8428FD028
:1057EC002A464432DC48DD4904F032FDDC4A1069BB
:1057FC00002819D03899515C022907D32A4648321F
:10580C00D548D64904F024FDD54A10692799884219
:10581C000AD1D069401E082806D32A464C32CE48FD
:10582C00CE4904F015FDCE4A3898105C012809D1F8
:10583C00907E012806D12A465232C748C74904F047
:10584C0007FDC74A906D002800D0D7E024970027A9
:10585C00469745971068C349884200D0CAE0C249B0
:10586C00C8682043C860C8682040419041980868C7
:10587C000125284308600868284041904198086831
:10588C00022210430860086817921040419041981A
:10589C00449703264396E020429042AC219821463F
:1058AC00FEF706FB44971596439618954295AF481C
:1058BC002146FEF7FDFAAE4E376280200521AD4A37
:1058CC00121D32607160B760F7603061329971619E
:1058DC002E99B1613899F161306A2299C841042836
:1058EC0004D39D48A449A82204F0B2FC70683E2859
:1058FC0004D39948A049AA2204F0AAFC25211798A0
:10590C00169170549D481030356829680140296003
:10591C009B488030B0649B482818142104F03EFB4F
:10592C00800097494118306417917164E8B20838C7
:10593C00142104F033FB20990840189C2146814027
:10594C00F164B068F26802433369134372691A4315
:10595C00B3691343F2691A43336A13432A681A432F
:10596C002A602546A203904218D10020179A106095
:10597C007060854A11600346014628E0389C20027D
:10598C002EE52A463A327448744904F061FC744A94
:10599C002898105C022800D384E68AE67068C4B2AA
:1059AC00179A1460784A1160401E032838463B460B
:1059BC0039460CD8611E88001018C367159B0B4024
:1059CC0029469940714B19607C30BC321346F76301
:1059DC00169AB5542422B75430657365B165604A84
:1059EC001665B2626A4B586835998843586028032B
:1059FC006849086054201754D765249F3B980507C5
:105A0C001468A068C00026D4A068634901402943EB
:105A1C00A16062480068624904F0C0FA40003C9002
:105A2C003C98002817D03C98401E3C903C9800288D
:105A3C0011D03C98401E3C903C9800280BD03C98D0
:105A4C00401E3C903C98002805D03C98401E3C9051
:105A5C003C980028E7D1A0682840369B07D1404DE0
:105A6C00A96D1943A965E96D01220A43EA65A1688C
:105A7C002C9A11403A4DAA6D1A405118AA6D68D152
:105A8C0024972999C9432091F33918910A40921C03
:105A9C00AA65A268D2072E4630D1E26818239A4331
:105AAC00B3681343E3602B99725C521E534253410B
:105ABC00726823991140356C0D43776C2F43B56C8C
:105ACC003D43F16C294319432369364D1D400D4369
:105ADC0025610123DD07AA4226910ED00325AD07CF
:105AEC00AA420AD09B079A4207D0299B9B041A40D2
:105AFC002D4D2F689F43BA182A60194E326B531ED6
:105B0C009A411203337E9B03757EEF031F43B57ED0
:105B1C006B033B43F7681F4317433369002B23493F
:105B2C0002DA17311940279127990F430C49289A0B
:105B3C008A5C52003A43389E8F5D012F3AD1002D7A
:105B4C0036D007498D6D35438D65CD6D2F43CF65AF
:105B5C0030E01A43AA659BE071C0000814BE00082F
:105B6C00640A00200024014034100240000400505C
:105B7C00C80A002004000240E6BE0008FF7FFFFFB9
:105B8C0000080240F8FFFDBF8408024044090240AF
:105B9C0008E400E000E100E0E8FFFF6F5C0B002090
:105BAC00400D030002FCFF1F08270140E8FFFF7FA8
:105BBC001E9D2A43F34E756A002D05D0379F613721
:105BCC003D401543B26A2A43E568EF4F2F40174317
:105BDC00E7602569ED4F2F4026990F4327616569D2
:105BEC002F9FBD43776B2F436761656970212891A7
:105BFC008D43B76B3F012F436761002B13D03B994B
:105C0C004D05AB421ED1DF4B1B6E1D46299E354008
:105C1C000F2DA56A0CD0F0271F40F02F08D120992A
:105C2C000D43A5620EE0A36A20990B43A36209E021
:105C3C00D44DED69AD001C351C272F402099B9407F
:105C4C001943A162E168D24B0B40934215D1002756
:105C5C00CC4BDF65996D3B9A1143259A914399651D
:105C6C00002815D03F973E97CA483D903DA8FDF7B8
:105C7C0005FB00280ED072B6FEE7C24A906D36992D
:105C8C000843259988439065D06D3B990843D065AE
:105C9C0072B6FEE72C983E90BF483D903DA8FDF7AC
:105CAC00EDFA002801D072B6FEE72A983E90BB4868
:105CBC003D903DA8FDF7E2FA002801D072B6FEE750
:105CCC0022983E90B6483D903DA8FDF7D7FA0028A3
:105CDC0001D072B6FEE7B349B34D8F65CF653A98E4
:105CEC0004048D63CF630F643E464F64349888641C
:105CFC001D98C8640C651C98486508463830279078
:105D0C00FDF7E6FC002801D072B6FEE7A749802219
:105D1C000E624E62281D41C10E604E603498886040
:105D2C00269208390846143054C00846FDF7D0FCBA
:105D3C00002801D072B6FEE79D489A49C860087CDD
:105D4C0000281DD19749487446904590994B996805
:105D5C00249A11439960996811403D913D991968B5
:105D6C00012211431960196811403D9144900320A0
:105D7C004390369842903D9842A92198FEF798F8A6
:105D8C00259888490874CE613B980874487C012892
:105D9C0001D172B6FEE72598824B1874D868C16B96
:105DAC003B9C21432D9A9143C1630168824A114067
:105DBC0001608249FE3902680A4002600168C02213
:105DCC00914301605E741C741E98401E7C4A774996
:105DDC000A634E638E63C8630E644E648E64409691
:105DEC003F963E963D962698802805D0379A3E3AA7
:105DFC007448754904F02CFA6D216C480F46405CD0
:105E0C00002822D16C21694A5054116B6C4A914282
:105E1C001BD10121CA02674CE3681343E360E368BA
:105E2C0013404293429A22680A43226022680A4035
:105E3C004192022146914590449043913298429070
:105E4C00419842A92198FEF733F825985749C8552F
:105E5C00086B02683B9989072091884205D0584904
:105E6C00884202D05949884205D128998A434F4922
:105E7C00896B114300E01146554A904209DD554AA1
:105E8C00904211DC4E4A904214D0534A904211D0A9
:105E9C0070E00122920790420CD04C4A904209D0FB
:105EAC004E4A904206D065E04D4A904202D04D4A8F
:105EBC0090425FD14C4A11403C4A126C0A432699DD
:105ECC008A433A4B996C11430160D96BC162596B8F
:105EDC008162464941181B9AD141072907D83B9A40
:105EEC008A40E1210A4202D03049496C01633B9A55
:105EFC00426178232D491793CA546E231693CA54C2
:105F0C000B466E335A709A70DA701A711D465A71BC
:105F1C0074231493CA540B4674335A709A701593A5
:105F2C00DA70CA556C222392895C012901D172B6B0
:105F3C00FEE725991D4AD1553B99239BD154816885
:105F4C002B4A0A4082602B4CA0420ADD2A49884227
:105F5C0012DD214988425AD02249884257D0204923
:105F6C0052E0264988424BDC0121890788424ED0F9
:105F7C00164949E00A46A2E71849884247D0104919
:105F8C0042E0C046640A00201902FEFF02FCFFDF5B
:105F9C00E7FF3F8320000014400000188000001C25
:105FAC000001002000000020000201406C090020CC
:105FBC000074004034100240FFBFFFFFFFF0FFFFF2
:105FCC00002C014071C000084FBF000800040040C5
:105FDC00FF2B0140FF4301400040014000200040E6
:105FEC000048014000440140FFFCFFFF00D4FEBF0D
:105FFC008800CEFFFF1F0040FF3F0140FF0F004015
:10600C00F649884203D0F649884200D084E1F5492C
:10601C00239A8E543B9ACA55A0420ADDF249884213
:10602C0010DDF249884219D0F149884216D0F14965
:10603C0011E0F14988420ADC0121890788420DD020
:10604C00EE4908E0EE49884208D0EE4903E0E34906
:10605C00884203D0E249884200D065E1E148806B78
:10606C002C99C841062800D9CBE03B998140572098
:10607C00014200D1C5E0DB48006C00280DD03B99F3
:10608C000902884209D03499884206D03B98C20252
:10609C00623ADD48DD4904F0DBF8D248806C269981
:1060AC000843802806D03B98C202613AD648D749AB
:1060BC0004F0CEF8CB48C05D002802D1C949239A20
:1060CC0088542598C749C855086B2099884202689E
:1060DC0005D0CC49884202D0C849884205D12899BC
:1060EC008A43C049896B114300E01146C84A90426B
:1060FC0009DDC84A904211DCC24A904215D0BB4A15
:10610C00904212D006E10122920790420DD0BB4A78
:10611C0090420AD0BA4A904207D0FBE0B54A90426E
:10612C0003D0B34A904200D0F4E0BB4A1140AD4AD0
:10613C00126C0A4326998A43AA4B996C114301604D
:10614C00D96BC162596B8162B44941181B9AD14118
:10615C00072907D83B9A8A40E1210A4202D0A1497B
:10616C00496C01633B9A42619E49179BCA54169B2A
:10617C00CA546A70AA70EA702A716A71149BCA5464
:10618C00159B5A709A70DA70CA55A149884205DC81
:10619C000121890788420DD0984903E0994988422A
:1061AC0008D09249884205D09D4AA5329648974915
:1061BC0004F04EF88B482399405C012801D172B64B
:1061CC00FEE725988749C8553B98239A8854086B55
:1061DC008168944A0A40543282608D49884207DDB6
:1061EC008C4988421ADC8749884222D07F4919E0C1
:1061FC000121890788421CD08049884219D08049E6
:10620C0010E00120C202633A7F48804904F020F874
:10621C007448006C002800D031E73EE7744988428E
:10622C0007D07449884204D0774878497E4A04F0F4
:10623C000FF86C4B23981E54186B016A026A3B9D35
:10624C00AA4302628269F0242C94A2438261259AAB
:10625C0011432A9A91430162C1681D9A9143C1600E
:10626C00C168724A1140C160DD557149884208DC31
:10627C000121890788420DD0604988420AD05749CC
:10628C0006E05749884205D05E49884202D05749FA
:10629C00884259D125985349C855239A8D54086B77
:1062AC0042685849884201D162490A4028998A4378
:1062BC0081684260564A904205DC01229207904266
:1062CC0007D04E4A03E0494A904202D04D4A9042D0
:1062DC0002D180229143816042483146239A8654F0
:1062EC00C55540963F963E9525983D903DA8FEF7A6
:1062FC004DF8002801D072B6FEE73A48006B4449CD
:10630C00884218DD434988422BDC3E49884234D010
:10631C0036492AE00A460DE73B483C49404A03F01F
:10632C0097FF3048006B72E6D202643A3648374920
:10633C0003F08EFF92E60121890788421DD02F4978
:10634C0088421AD02E4910E0EA02923A2E483A4975
:10635C0003F07EFF23482399405C01289AD172B642
:10636C00FEE72349884208D02249884205D0334AA7
:10637C00C83A2548304903F06BFF1A482399405C12
:10638C00012801D172B6FEE716484654006B816EA7
:10639C0029430E222892914381663D963DA8042103
:1063AC001591FDF7F3FF002801D072B6FEE70D48FA
:1063BC00006B1749884207DD1649884240DC1149B9
:1063CC00884249D009493FE001218907884243D0DE
:1063DC000A49884240D00A4936E0C04600100040C5
:1063EC00001400406C090020FF3F014000400140B8
:1063FC000044014000480140FF0F004000040040F1
:10640C0000200040002C014071C000084FBF000864
:10641C00FF2B0140FF430140FFFCFFFF00D4FEBFF8
:10642C00D914000088FFCEFF6C1C0000FFBFFFFFDB
:10643C00FF1300408FFF0FFFCCC20008C4090000FF
:10644C00EC49884208D0EC49884205D0EB4AC83A5E
:10645C00EB48EC4903F0FCFEEB482399405C012827
:10646C0001D172B6FEE7E8484654006B816EE74AEC
:10647C001140329A11438166E549E64A0E624E623A
:10648C008E624B20179000020A6048601A98886050
:10649C00CE602E980861229848618E61CE6184206E
:1064AC000B900858002836D180200025D8490D546F
:1064BC00086890422FD10124A003D74AD168014328
:1064CC00D160D1680140429142981068204310601D
:1064DC00106820403D90469445954495022743977B
:1064EC000920400242903D9842A923912198FDF742
:1064FC00DFFC46944595449443972E9842902198FE
:10650C002399FDF7D5FCC54A1069C54908401061AF
:10651C00E006C44908602422BD480B9907924250FA
:10652C00006801683B9A91430160FEF75BF8012813
:10653C001BD0B748806A002801D0FEF7CFFA3B9BEE
:10654C009903B348006882680A43826081681C9A88
:10655C00914381600168B44A0A40026001681943A2
:10656C000160FEF7B7FB002801D072B6FEE7A84821
:10657C000068AE4988420BD0AD49884208D0A54985
:10658C00884205D0349A62329D48AA4903F060FED5
:10659C0026989F49085C012801D172B6FEE79C4AF7
:1065AC000B9807991150146820682E9020683B9B1B
:1065BC00984320602498401EA1680140A160506E51
:1065CC0023900028184612D0A568A068400F9A4F57
:1065DC00395C9A4A105CC00003F0E0FC3B90280147
:1065EC00400F395C954A105CC00003F0D7FC68275B
:1065FC008749C8536A223B982092885226980E5499
:10660C002E98206038980B9A88508848844216D06F
:10661C008748844213D07F48844210D0349A9332F6
:10662C007748844903F014FE26987949085C0128C0
:10663C0001D172B6FEE77648416E23910468744826
:10664C000B99079A425020683B9020680125A8437B
:10665C0020602F984006A1688143A16023980028F0
:10666C00284615D0A0682E90A068400F7249095C8E
:10667C00724A105CC00003F091FC05462E98000194
:10668C00400F6D49095C6D4A105CC00003F086FC3C
:10669C005F49C85320980D5226980E543B982060A1
:1066AC0038980B9A88506148844214D060488442D0
:1066BC0011D0584884420ED0349A343250485D4937
:1066CC0003F0C6FD26985249085C012801D172B628
:1066DC00FEE74F4804684E4A0B9B0798D050206841
:1066EC0021680125A94321600C9569078843206026
:1066FC003898D0502698165456665148406A5049DE
:10670C00496A091A64290ED84D49496A091A64293B
:10671C0009D84B49496A091A642904D84849496A75
:10672C00091A6529EBD3E6204649474D14900D52C2
:10673C00E022464813928850A81CE42212928852F8
:10674C003A9888810C9888606720088040480478C3
:10675C00012C01D03F4800E03F4803F079FD0C9834
:10676C008704012C3D4C00D1C5E03D4803F070FD81
:10677C0002F0D2F93B4803F06BFD3B490E86CE8507
:10678C008E854E858E840E84681C08853748488417
:10679C00CD8437484069002805D53648344988608F
:1067AC003548886048692648406A31994018304914
:1067BC0009691E9A114261D02149496A814265D208
:1067CC002B490969114259D01D49496A81425DD250
:1067DC0027490969114251D01949496A814255D258
:1067EC0023490969114249D01549496A8142DED3CE
:1067FC004CE0C0460044014000480140C409000080
:10680C0071C00008CCC200086C090020FFF0FFFF2B
:10681C00DC080020003801403410024008E400E09D
:10682C00FFFFFF0000E100E0FFFF00FC0044004020
:10683C0000800040B8BF000840C3000838C30008FF
:10684C00E8090020FC060020FF7F00000000FFFF8D
:10685C0048F0010864BD0008F1C0000800F8010808
:10686C0025C00008E8C3000800000020FFFF00005E
:10687C000020024023016745AB89EFCDEB4B186933
:10688C00EB494A1C1A61084200D143E1E7484069D0
:10689C00C00704D0E54A50690C99884350613F20E9
:1068AC00E449886433980874087542A8FDF71EFA09
:1068BC00002801D0E0481CE0E048026A436A204608
:1068CC00FDF75CF9002813D1DC48826AC36A2046C4
:1068DC000830FDF753F900280AD1D848026B436BF6
:1068EC0020461030FDF74AF9002801D101F056FF7F
:1068FC00D34803F0ADFCD3480069000704D4D24858
:10690C0003F0A6FC02F008F9D04803F0A1FC02F059
:10691C00EDF920783899C94A5054104620306178E6
:10692C004170A1788170E178C17021790171617930
:10693C004171A1798171E179C171217A0172617A18
:10694C004172A17A8172E17AC172217B0173617B00
:10695C004173A17B8173E17BC173217C0174617CE8
:10696C004174A17C8174E17CC174217D0175617DD0
:10697C004175A17D8175E17DC1750C990D02118C5C
:10698C00B34B069559538188139A9952129A99527E
:10699C004188E22211929952C188149A995221216C
:1069AC000391CA00C18910929952832100914A0027
:1069BC00018A0F92995241218A0041890E92995273
:1069CC008121490080890D915852188B00283BD1A8
:1069DC006420319A643A97498865CA65496E0029E2
:1069EC0000D01046934A1066484248415066994A76
:1069FC00101F0A9000680104159D2840394040186A
:106A0C00684010600C981060259810600026304685
:106A1C00FDF7B0FB2846FDF7ADFB4296874CE068CE
:106A2C004290429808304290429806608A4803F09F
:106A3C000FFC607C012844D188489BE0711C844881
:106A4C00008B0E468142C3D22A9882490860844842
:106A5C001D9901607748406A7649496A091A379A44
:106A6C0091420ED27349496A091A914209D271496D
:106A7C00496A091A914204D26E49496A091A91422B
:106A8C00EAD32A987349086175481D990161002061
:106A9C00684908654865486A6649496A091A914215
:106AAC00CCD26449496A091A9142C7D26149496AF0
:106ABC00091A9142C2D25F49496A091A9142EBD331
:106ACC00BCE725985D490874C86801680C9A1143A5
:106ADC00016001683E220A40022A03D141680C9AE7
:106AEC0011434160554846740C9901745D4803F09C
:106AFC00AFFB2798FCF7E6FF002801D05A4839E095
:106B0C005A4803F0A5FB5A48FCF7DCFF00282DD0AF
:106B1C0058482FE04748406A319940184349096961
:106B2C00394200D1B2E64349496A814200D3ADE60D
:106B3C003E490969394200D1A8E63E49496A814279
:106B4C0000D3A3E639490969394200D19EE6394997
:106B5C00496A814200D399E634490969394200D126
:106B6C0094E63449496A8142D8D38FE6424803F00F
:106B7C006FFB424803F06CFB429641480068414968
:106B8C00884204D0404841496F2203F061FB5420F5
:106B9C0016903B49085C012800D121E10C9816990C
:106BAC00374A5054106882688168C907339972D08B
:106BBC0025990A4033996ED181681F9A1140012999
:106BCC0029D18168324A1140259A114381603A9942
:106BDC0001601849496A8268D2075BD0154A526A2B
:106BEC00521A022A17D88268D20753D0114A526A15
:106BFC00521A022A0FD88268D2074BD00D4A526A19
:106C0C00521A022A07D88268D20743D0094A526A1C
:106C1C00521A032ADFD31A4B996D369A1143996590
:106C2C00D96D0C9A1143D965314634E000200240ED
:106C3C00FAC30000E809002017C10008000000207A
:106C4C00A6BD00080004005046BC000848C300085C
:106C5C00FC060020180C00509EC00008B3C00008B1
:106C6C0018080050A6BC000849B9000878C30008F1
:106C7C006C09002060B900088CC30008B8BC00087F
:106C8C00640A00200024014071C0000860C20008A2
:106C9C00E8FFFF7F33998268D207F24A926D40D1A8
:106CAC00189B1A40259B1A43FB4B9A65C268C36814
:106CBC003A9DAB43C360F94B183384681C43846022
:106CCC002A40F74B8468002C2ED5429C641C4294BD
:106CDC00429C9C421AD88468002C25D5429C641C8A
:106CEC004294429C9C4211D88468002C1CD5429C36
:106CFC00641C4294429C9C4208D88468002C13D596
:106D0C00429C641C4294429C9C42DBD91698E24AF9
:106D1C001654906D36990843259988439065E1483F
:106D2C005FE13698024308E0C3681343C360DA4856
:106D3C00826D0C980243259882431698D64B1E54AC
:106D4C009A6500294CD0D84803F082FAD2480068E2
:106D5C00D649884208D0309AAF32D548D54903F08D
:106D6C0077FACD4800681990199881681698CA4A24
:106D7C00105C421E504250414907339900D40146E1
:106D8C00002900D02CE10C981699C34A505419983C
:106D9C00C068C0070FD119988068C00706D0199A2F
:106DAC009068BE490840259908439060199AD068AC
:106DBC000C990843D060429619988068C00744D15A
:106DCC00B6482F301999896801420BD0B24A906DA0
:106DDC00369908439065D06D0C990843D065FFE057
:106DEC00B048FEE0199A9068AC4908400C990843E9
:106DFC009060B1480068000221D5B0480068B049E5
:106E0C0003F0CCF8401C42904298002817D04298CE
:106E1C00401E42904298002811D04298401E429049
:106E2C00429800280BD04298401E4290429800286D
:106E3C0005D04298401E429042980028E7D19648CF
:106E4C00407E012801D001F0B8FC1698924A1654E5
:106E5C009C48401E916D0140329801439165D66566
:106E6C001C23199D2B60106D9749984A984CC4624D
:106E7C00026341636968369A114369600799415C02
:106E8C00012900D1A6E0014624310C9A0A704A78F7
:106E9C00012A00D09BE0259A4A70C66301680A68F3
:106EAC000C9CA2430A60826CC46C5460026D002A74
:106EBC0002D0446D856D6560199C4034056C1D4095
:106ECC000C9BAB40834D2F681F432F60159B4B6071
:106EDC008568814B102D1F4600D027468F60102DE2
:106EEC0000D01C46CC600B68289C23430B60406C84
:106EFC0003681E9C234203D00368329C2343036027
:106F0C00002A03D01068329B1843106008680C9A52
:106F1C0010430860199A9068604908401599084315
:106F2C0090606E4803F094F96D48806E3B90632836
:106F3C0001D901F022FC6A48C06E309006E0684826
:106F4C0006773B98642801D301F017FC6448046F62
:106F5C00002CF4D0634BDC88DD88634A55432D0C40
:106F6C009B277F006149CD535D48456FEF08ED1BB2
:106F7C002C193294E50855432D0CC827CD53856F39
:106F8C00EF08ED1B1F891C46ED19EF08584A5743B3
:106F9C003F0C584BFF18CA23CF5221462368DF08F9
:106FAC00DB1BA788DB19DF0857433F0C1B9A5743A1
:106FBC00309ABF1ACC224D4CA7523B9A521C3B9292
:106FCC0082660667329A426785670B60B7E70E7078
:106FDC002699C163A8683149084015990843A860EF
:106FEC00454803F035F94148818A006902F0D2F92D
:106FFC00424801460C39424A0A60424A0A6002463B
:10700C00083A002327931360031F1A9A521E1A6022
:10701C00334B5B6A0468002C1ED0314C646AE41A52
:10702C00302C17D80468002C16D02D4C646AE41A46
:10703C00302C0FD80468002C0ED0294C646AE41A4A
:10704C00302C07D80468002C06D0254C646AE41A4E
:10705C00302CDFD972B6FEE74368934204D12A483C
:10706C00086002E0640A00204260179880000890D3
:10707C000B200290400228900C98C10418918105B5
:10708C000991C1050191C00604902048FE3005907D
:10709C0027982390209048E0640A0020E8FFFF7FA7
:1070AC00FFF1020000C4000844C1000800240140A4
:1070BC0071C0000814BE0008082701405C0B0020BA
:1070CC00400D0300FFF0FFFF7FB70008CDB30008B1
:1070DC00153200080400024004000020FCB900082E
:1070EC00E80900200000002088130000FC060020A6
:1070FC00C4090000A8FD000065C100080C30004068
:10710C00CCCC000055550000AAAA0000D9140000F0
:10711C000020EB493B9A88500875EA4803F098F830
:10712C00E74800688821222242502798401CE649F3
:10713C00496A814245D3E448006D002821D0401EA5
:10714C00E14908651DD1E048406DE049012800D1B6
:10715C0010312A9A0A60DE49012800D110311D9A9B
:10716C000A60411E4A1E9141D74A5165127E002A7F
:10717C00319900D10021012801D0D348C16CD248EB
:10718C000165D148006E002818D0401ECE49086613
:10719C0014D1CD48406ECD49012800D11031159A3B
:1071AC000A60411E4A1E9141C74A5166012801D00E
:1071BC00C84800E0C8480068C3490866C248406A2D
:1071CC0027902398401CC049496A814201D200F0A3
:1071DC0077FDBD48416A2391006F00283ED0BF4D1A
:1071EC00E888E988BE4B5943090C9B225200BD4CE0
:1071FC00A1522646B44F796FCA08891A08183B90D9
:10720C00C1085943090CC822A152B96FCA08891A7E
:10721C002C462A898A18D108B34D6943090CB34B03
:10722C00C918CA23F15223682646DC081B1BB488F4
:10723C001B19DC086C43240C1B9D6C43BD6EFE6E4D
:10724C00A41BCC26A74884536C1CBC6600243C674A
:10725C003B987867BA67A148036002E0CA20A1494D
:10726C00095A48209F4F385E0CB2201A0A2102F0AE
:10727C006DFE4A21795A41433A8D8918EA221C92B3
:10728C00B9524C21795A41437A8D8918EC221992C2
:10729C00B9524E21795A4143BA8D8918EE22B9520E
:1072AC005022BA5A4243FB8DD3182C9A3093BB52BE
:1072BC005222BA5A42433B8ED218F2231E93FA52F0
:1072CC00169ABA5A42437B8ED218F4232E93FA5252
:1072DC005622BA5A4243BB8ED318F622BB525822BE
:1072EC00BA5A4243FD8E5619F822BE525A22BA5A45
:1072FC0042434620385A1018FA22B852FC22BA5A85
:10730C00002A02D1E822774DA8523998754A105EAE
:10731C00844203DDCE200122724D2A523A20714A5A
:10732C00105E844203DACE2000226E4D2A522B9836
:10733C006C4A105E844203DAD0200122694D2A5235
:10734C003E20684A105E844203DDD0200022654D49
:10735C002A521D98634A105E844203DAD22001221D
:10736C00604D2A5242205F4A105E844203DDD220D7
:10737C0000225C4C2252C8225A483B92825A98B244
:10738C00824206D3B0B2824203D8D420554B1B5A4A
:10739C0008E0B0B2824201D9002300E00123D420DE
:1073AC00504C2352CE244F483294065B701E4442FC
:1073BC00444188B28242339800D82046D0244949AF
:1073CC00095B4F1E7D427D410028339800D1284631
:1073DC005F1E7D427D410028339806D1012D06D0D9
:1073EC00309880B2824217D325E00128F8D10220D0
:1073FC0036490861DE2001213A4A1152D420135A31
:10740C00115B3298165A2C98105A30903B98125A9D
:10741C00309880B282420ED2002E0CD100290AD1B3
:10742C00002B08D1022029490860DE2000212D4ABA
:10743C0011523B98125A2B481E99405A824213D231
:10744C00214B986B31994018596A81420CD3D62143
:10745C00244C635A4420205A834202D2581C214B9C
:10746C0058521949486A88631E4D3298285A401E52
:10747C00444244414421685AD623ED5A8542339EF6
:10748C0000D02646D2251748405B441E604260411E
:10749C00002E339C00D10446012C07D101200B4A4D
:1074AC001061DC220F4CA0523B98225A0D482E9CA6
:1074BC00005B82421CD900220A48C2521AE0C04624
:1074CC00C004002013BA0008E8090020180C005072
:1074DC0018080050400A0020440A00200000002038
:1074EC0088130000FC060020C4090000A8FD000061
:1074FC00FC48C25A002A0FD1FA48329A805A002806
:10750C000AD1FE48405B002806D10120FC4A1060DD
:10751C00DC200022F94C2252FE22F8483092805A8C
:10752C0002282AD1F748406C012800D1F4E03398A6
:10753C00F44A10760A98006801042A9B1840189C9B
:10754C00214040185840EE490860EF49D164506D15
:10755C00002800D03199EB4A1165414241415165F7
:10756C00EA4A101F006801041D9B1840099C214029
:10757C004018584010600120CCE0C01E01282AD8C9
:10758C00E048406C022800D1C6E03398DD4A107602
:10759C000A98006801042A9B1840189C2140401846
:1075AC005840D7490860DA49D164506D002800D0A2
:1075BC003199D44A1165414241415165D34A101F5A
:1075CC00006801041D9B1840099C2140401858403C
:1075DC00106025989EE0C948329A805A01282AD119
:1075EC00C848406C032800D196E03398C54A107601
:1075FC000A98006801042A9B1840189C21404018E6
:10760C005840BF490860C349D164506D002800D070
:10761C003199BC4A1165414241415165BB4A101F29
:10762C00006801041D9B1840099C214040185840DB
:10763C0010603A986EE0B14A3B98105A1C9C125B51
:10764C00904225D9AF48406C042865D03398AD4A98
:10765C0010760A98006801042A9B1840189C214057
:10766C0040185840A64908603198D0641065506D98
:10767C00414241415165A54A101F006801041D9B00
:10768C001840099C2140401858401060159841E062
:10769C009A4A199C125B904232D29A48406C052847
:1076AC0023D03398974C20760A98006802042A9DC0
:1076BC002840189E324080186840914A10609622EB
:1076CC00E264606D002800D0319A8E4C22654242F3
:1076DC00424162658D4C201F006802041D9D2840AC
:1076EC00099E324080186840206085480C9A0261DF
:1076FC00DC20259A814C2252605AE0521F9809E0F6
:10770C002A987F49086181481D99016100207D49B3
:10771C00086548657B4948647A48007B002809D194
:10772C002C9876490D5A3B980E5A0020AE4205D241
:10773C000C9D12D2002500281ED010E06F49069A2D
:10774C00885A401C885233986E4F3873724802F036
:10775C007FFD387BAE420C9DECD300280CD06749E2
:10776C002E98085A3B9A895A814205D86B4802F0E8
:10777C006FFD0020634908736249C86B684A801822
:10778C00496A8142339802D25E48007FC043C007E9
:10779C0000D188E033985B490877486AC863614830
:1077AC0002F056FD55483B99415A119A805A814234
:1077BC0007D2524CA1525C4802F04AFD3B98215A28
:1077CC00339D4E48139A805A814205D94B488152B9
:1077DC00564802F03DFD339DCA26484A915F1498E5
:1077EC00105E814207DA1498444C2152504802F042
:1077FC002FFDA15B339D4148129A805E0AB28242F2
:10780C0008DD3E4C129821524A48114602F020FDE8
:10781C00A15B339D3998394A105E323009B28842E7
:10782C000EDA36480E9A805A434A904208D0401CD1
:10783C00324C0E9AA0523F4802F00AFDA15F339DD4
:10784C001D982E4A105E323888420ADD2B480D995D
:10785C00405A3949884204D0401C28490D9A885214
:10786C00339D26493B98085A498D643981420ADD7B
:10787C0022490F9A895A304A914204D0491C1F4A16
:10788C000F9BD152339D1D49098D643181420AD21F
:10789C001A481099405A2849884204D0401C17496C
:1078AC00109A8852339D1749086C244A8018496AEB
:1078BC00814209D31349486A0864214802F0C8FC84
:1078CC00002D01D001F0A4FC1E48056B1E4885421A
:1078DC000ADD1E48854243DC1D4885424DD01D48BB
:1078EC0042E0C046FC06002001208007854244D0BF
:1078FC001948854241D0194836E0C046FC060020A4
:10790C00180C0050E8090020581B00001808005003
:10791C0088130000B80B0000D9B9000800BD00089E
:10792C0060EA000016BD000830BD00084ABD000822
:10793C00A0C30008B8C30008FFFF000080EE3600AB
:10794C00D0C300086C090020FF2B0140FF4301400D
:10795C00002C014000400140000400400020004089
:10796C00F348854209D0F348854206D0F248F349E2
:10797C00059A02F06DFCF248056B6C6BF148854280
:10798C0005DC0120800785420FD0EF4803E0EF486B
:10799C0085420AD0EE48854207D0289A1F3AE6481D
:1079AC00E64902F055FCE648056BAE6B97204000AB
:1079BC00E84F3E52A01B17998900785202F08EF9BD
:1079CC000446304602F08AF90146204602F098F847
:1079DC00014601F097FF06463B98385A02F07EF9B3
:1079EC00314602F031F802F02FF90A2132902E9133
:1079FC0002F0D4FA132109017852D8203B90385A5E
:107A0C00002810D0696AD448C06A379A95329142DE
:107A1C000CD9D049309A895A002907D1CE4A117213
:107A2C00401CD06207E0CB484018B2E0002829D0B7
:107A3C00401EC949C862642824D3C84802F008FC17
:107A4C0000254595449501204390389F42974695D3
:107A5C0042AEC34C20463146FCF72AFAA7622F9857
:107A6C0046904595449502204390429720463146D6
:107A7C00FCF71EFAB849CD6233980872086B401CAB
:107A8C00086301E0B448006B0A281CD90025B149F1
:107A9C003B980D524295B348C068429042980830CA
:107AAC004290429805600420309A8852AE4802F009
:107ABC00CFFBA9490D63486B401C48633199491EA3
:107ACC0088420DD80FE0A44A516B491C5163319A7E
:107ADC00521E914207D9002802D0401E9E490863CD
:107AEC0000209D494863992045009A48415B9A487B
:107AFC00007A9E4A329B934203D3002801D0012284
:107B0C0002E000299A4A1BD08918924A515389B233
:107B1C00652915D300268F4C3B98265242969148E6
:107B2C00C068429042980830429042980660022009
:107B3C00309960528F4802F08BFB66538648007A6E
:107B4C004D218D008C49329A8A428249495B03D877
:107B5C00002801D0012002E0002985481BD008181C
:107B6C007C49485380B2652815D30020794C3B9949
:107B7C00605242907B49C9684291429908314291C6
:107B8C00429908600320309960527C4802F060FBF7
:107B9C006019002101807A4840680028339904D08C
:107BAC00401E7749486041424141DA256948405BB3
:107BBC0000285ED100295CD071482E994160E820E4
:107BCC00644B1A5A9B2149005B5A934229D9614C48
:107BDC003B9EA65B6B4CA64223D25E4C309FE75B70
:107BEC00002F1ED1721C5B4B3B9C1A53089B5B1ED7
:107BFC009BB29E4207D2574A089C3B9BD452002210
:107C0C00554B1A63224600234293564BDB68429332
:107C1C00429B0833429392B2429B1A604D4B1A5AC4
:107C2C005B5A934223D24B483B99405A00281ED0B2
:107C3C00411E8AB20020089B9A42024600D30A4693
:107C4C0044493B9BCA52429096B249480E388642F0
:107C5C0005D3319A893A38484B4902F0F9FA414830
:107C6C00C068429042980830429042980660394869
:107C7C00405B012813D137483B99405A414988420F
:107C8C0010D23449309A895A00290BD14291354986
:107C9C00C9684291429908314291429908602D4835
:107CAC003B99405A31996439642200280B4600D024
:107CBC001346294CE365002800D00A462648826505
:107CCC002548406A209988420DD92349886A496A17
:107CDC002091002807D0401E1F49886203D1FC2048
:107CEC0000211C4A115226202E901A48408B002845
:107CFC0000D19AE125492E9A895C002900D094E1A3
:107D0C00411E062946D849007944898849008F4488
:107D1C0006004C005C00270562007C0091001C48AA
:107D2C0002F096FA0020014601F036F97AE1C046DD
:107D3C00004401400048014071C000084FBF0008DA
:107D4C006C090020FF2B014000040040002C014076
:107D5C0000400140FC060020E8090020C8C00008D3
:107D6C00000400500000002077B90008A1090100B0
:107D7C00FFFF0000A2B900080F270000CABC0008D2
:107D8C005C0B0020DC0500007DBE0008C004002058
:107D9C0060BC0008F849884266D1F84802F058FAED
:107DAC000021339801F0F8F83CE1F54802F050FA64
:107DBC00F4480068F44988425CDDF449884267D095
:107DCC00F349884264D0F34958E0F34802F040FA92
:107DDC0000F0A2FE26E1F14802F03AFA6224F048E3
:107DEC00015BF048008C814209D10020339901F0ED
:107DFC00D3F86420EA49085A0853EA490884411E1A
:107E0C0088415E21E64A50520CE1E74802F020FA24
:107E1C006220E349085AE349098C884226D10120A3
:107E2C0000020021DE4A115010180181416001F05E
:107E3C00EFF9F7E0DD4802F00BFA6220D849085A56
:107E4C00D849098C884211D1CA20D54A105A1499A4
:107E5C00505212995052C820105A119950521399DD
:107E6C00505201F0D5F9DDE0D14800E0D14802F0E4
:107E7C00EFF9D7E0D04988420AD0D049884207D0E0
:107E8C00349A7432CE48CF4902F0E2F9BD4800680A
:107E9C00BC490B9A079B8B50016801221C929143A1
:107EAC00016000210160416019918160B9498842EB
:107EBC0000D0A7E0C449C868C44A1040C86002207A
:107ECC003B90042032902A983090199D24E03B98E6
:107EDC008140219F3868084338601C20329B184031
:107EEC00299B8340E80880003818046A9C4304628C
:107EFC00B8688843B860786890437860F8688843BD
:107F0C00F8601E98851C3298083032903B98001D02
:107F1C003B903098103030901C9EAE4031462898E3
:107F2C0001403BD030980838369A1040299A82404C
:107F3C0003202B468343A64CE3181C6E144211D12C
:107F4C006033A44F3C688C433C607C688C437C6001
:107F5C009F4F3C688C433C607C688C437C60196808
:107F6C00914319603B99891E8840219C21680143EB
:107F7C0021603299091F18220A4029999140EA0878
:107F8C009200A218136A8B431362A1688143A1600B
:107F9C006168B1436160E1688143E160681C0D2850
:107FAC0029D0401E02221E9082401046289908407B
:107FBC00A7D01821309B1940299B8B4003212C46BC
:107FCC008C43834F3C19276E1F4200D07FE76034EF
:107FDC00804E3768874337607768874377607C4F7C
:107FEC003F6887437A4E37607768874377602068AD
:107FFC00984320606BE7049877490860BFF34F8F74
:10800C00BFF36F8F8C205F49199A0A500B980A5056
:10801C0088200A5080200A54CA6661490869898AF6
:10802C0001F0B8F900205E4948836C48007D0028B7
:10803C0001D1FFF77AF84520C10068483B914058C0
:10804C00042801D8FFF764F8074627256348405DEC
:10805C00329001201E90C443B81E3090044000267C
:10806C005F4A03E0B61CB44200D1BDE05B48801906
:10807C00415D51408AB25208C9071DD059494A4046
:10808C005308D1071BD15A08D9071DD055494A406E
:10809C005308D1071BD15A08D9071DD051494A4062
:1080AC005308D1071BD15908DA071DD04D4A51404E
:1080BC004A08C9071BD11CE05308D107E3D0494932
:1080CC004B405A08D907E1D15308D107E3D04549B1
:1080DC004B405A08D907E1D15308D107E3D04149A5
:1080EC004B405908DA07E1D14A08C90701D03D498C
:1080FC004A402823C15C51404808C9071DD0394962
:10810C0048404108C0071BD14808C9071DD0354954
:10811C0048404108C0071BD14808C9071DD0314948
:10812C0048404108C0071BD14808C9071DD02D493C
:10813C0048404208C00795D01BE04108C007E3D077
:10814C00284841404808C907E1D14108C007E3D09D
:10815C00244841404808C907E1D14108C007E3D091
:10816C00204841404808C907E1D14208C00700D166
:10817C0078E71C48424075E73930000036C00008EB
:10818C0076BC0008DC080020FF4B0040004C00408F
:10819C0000800040003801405DB300084BC000086F
:1081AC00FC060020E809002090BC000858C3000819
:1081BC0060C000082AB90008004400400048004094
:1081CC0071C00008DCBB000834100240FFBFFFFF89
:1081DC00001802408018024080E100E0C00400203A
:1081EC00FFFF000001A00000F80742D0FD48001975
:1081FC00405D424090B24008D1071DD0FA4948403A
:10820C004108C0071BD14808C9071DD0F649484092
:10821C004108C0071BD14808C9071DD0F249484086
:10822C004108C0071BD14808C9071DD0EE4948407A
:10823C004208C0071BD11CE04108C007E3D0EA4844
:10824C0041404808C907E1D14108C007E3D0E648DE
:10825C0041404808C907E1D14108C007E3D0E248D2
:10826C0041404808C907E1D14208C00701D0DE48A7
:10827C004240791C48424841DC4C3099615C3D19C4
:10828C006D1E2D782D02691892B29142339900D14E
:10829C000146012903D1D64801F0DAFF25E0D54883
:1082AC00018B329D4A1B50425041002D339A00D015
:1082BC000246002A19D093204500CA4A30953298BC
:1082CC0050558B20850000201C955051D25C102AF3
:1082DC0012D0062A1AD0032A25D1329A002A2BD082
:1082EC00914229D08620029960E00020BD493B9A3A
:1082FC0088500875FEF714FF3298002828D0814268
:10830C0026D003270B2186261E9AAAE03298002835
:10831C002DD081422BD0359828308621B14A11546A
:10832C0002210B20C7E0AF48309940181E9981708C
:10833C0026994A4042703EE0637921790902CA18B5
:10834C0011467E397C25ED43A94222D203212CE033
:10835C00617920790002421810467C387A23DB437D
:10836C0003279026984228D21E9A394679E0E17864
:10837C00A078000240189C2800D395E08D22920032
:10838C00984B9A58125C022A72D0002A77D19A48DC
:10839C0088E0E178A47824026118521814469D3CB8
:1083AC009B25ED43AC4218D2022100988D4A309B9C
:1083BC00D21891705070032782E0E378A078329045
:1083CC0000021993C418151928469D389B22D243D4
:1083DC0090421BD202211E9A43E0824D309C2C19F4
:1083EC005B00A37003236370359B2A33EB184C009E
:1083FC00804D2C19255C5D7025186D781D70801CC6
:10840C009B1C491C9142F5D3C71C59E06000794A6A
:10841C0010184722D200734B9F588D2292009A5805
:10842C002F3309E01E7806705E1E36784670801C6D
:10843C009B1C641CAC4208D2165D002EF7D0022E99
:10844C00F0D13E88002EEDD1F1E7F448309A801837
:10845C00199AC270329A8270369A4270042200269F
:10846C002D9FEE488018309A86548018417027E072
:10847C004722D200E94B9A581288002A11D04200A8
:10848C006079E34B98549A1823795370E34A309CE3
:10849C0012191371D170002191702D995170052111
:1084AC0009E0E14801F0D4FE359828308621DB4AFA
:1084BC00115402200146D94A5218309BD0544F1CFB
:1084CC0039461E9881433A460240D448309BC31823
:1084DC000C46D04D03E09B1CA41E00D18EE01878F6
:1084EC0068404508C0071DD0CB4845406E08E807DA
:1084FC001BD17508F0071DD0C74845406E08E8072A
:10850C001BD17508F0071DD0C34845406E08E8071D
:10851C001BD17008F5071DD0BF4D68404508C0073A
:10852C001BD11CE06E08E807E3D0BB484640750839
:10853C00F007E1D16E08E807E3D0B748464075086C
:10854C00F007E1D16E08E807E3D0B3484640700865
:10855C00F507E1D14508C00701D0AF4845405E782A
:10856C006E407008F5071DD0AB4D68404508C0073C
:10857C001BD16808ED071DD0A74D68404508C00702
:10858C001BD16808ED071DD0A34D68404508C007F6
:10859C001BD16808ED071DD09F4D68404508C007EA
:1085AC0099D01BE04508C007E3D09B4845406808BC
:1085BC00ED07E1D14508C007E3D09748454068086E
:1085CC00ED07E1D14508C007E3D093484540680862
:1085DC00ED07E1D14508C00700D17CE78E48454046
:1085EC0079E7C046C004002001A00000E704002089
:1085FC007EC10008FC06002024C40008002A43D0D9
:10860C00864840183099405C4540A8B24008E907BC
:10861C001DD0814948404108C0071BD14808C907F3
:10862C001DD07D4948404108C0071BD14808C907E7
:10863C001DD0794948404108C0071BD14808C907DB
:10864C001DD0754948404508C0071BD11CE04108A6
:10865C00C007E3D0704841404808C907E1D1410840
:10866C00C007E3D06C4841404808C907E1D1410834
:10867C00C007E3D0684841404808C907E1D1450824
:10868C00C00701D064484540290A644CE019309A6F
:10869C0085548018417022982E996054BB1C1C98EC
:1086AC00235098B2424242412068014680314C68C6
:1086BC00202C339C00D11446002C30D10A78012A8E
:1086CC002DD00546543584686B800022CA602B80FF
:1086DC00524B309D5B190365039B4B60436E249D8D
:1086EC00AB420DD11A9B9C4203D10369002B514B19
:1086FC0000D0514B0A7043670068083001990BE0B9
:10870C001A9B9C4203D10369002B484B00D0484B69
:10871C000A7043670068269902680A4302600020C9
:10872C003E4D3B9968506221394C615A334B1A8C3F
:10873C00891A4A424A41602162522875DA835C20C8
:10874C00205A002801D1FEF7F0FCFC21304A1E9B78
:10875C005352E8215052294838498162FEF7E5FC12
:10876C002F4801F075FDBFF34F8F234914392D4865
:10877C000860BFF34F8F00BFFDE723480168CA08AC
:10878C00891A828889180160C90820484843000C5E
:10879C001B9948431949C866FEF725FC194818303F
:1087AC00144A516901435161506915480069000729
:1087BC0001D4FEF7A4F8FEF7A7F81048406A199BFD
:1087CC0006E00E49496A091A032901D3FEF7FEFA9D
:1087DC0019990968C90701D0FEF737FB19998968FF
:1087EC00C907EED19968074A11400C9A1143996058
:1087FC00E7E7C0460020024020ED00E0E809002039
:10880C0000040050E8FFFF7F00000020C4090000B6
:10881C00FC060020FFFF000001A00000C0040020A7
:10882C0085B300080400FA0540C40008294E00086E
:10883C0093B70008CD4D0008CFB30008E0930400B7
:10884C000248416A491C41627047C046E809002051
:10885C00F0B583B03848001F0568384A14682068A2
:10886C0004260190304041424141106C1C230340CE
:10887C0037469F40384602952840424242410A43BF
:10888C0030D0009401200226019D2A4632405142EC
:10889C0051419E40029A1642074600D00F46002FC7
:1088AC0032D008210D4069426941DA40120700D5E7
:1088BC000846002826D124200021204C2154009A5F
:1088CC0010680E21884310600120014699401A4B14
:1088DC001A680A431A60E06325216054616B002911
:1088EC000ED10FE02068800602D42068B0432060CF
:1088FC0011490868384308601048016B002901D001
:10890C000E48884703B0F0BD2346206880060B4A0A
:10891C0006D418680A2188431860252001211154B7
:10892C002420002111540449086830430860D16A9E
:10893C000029E5D1E6E7C04604000240C80A002041
:10894C00F0B583B06E4D286801680291EF21CC0020
:10895C0047686C49884204D06B486C49224601F048
:10896C0077FC6869042806D0082804D0621C664885
:10897C00664901F06DFC02233846184041424141E2
:10898C0002981840424242410A4308D1A86DC006E1
:10899C0003D48834A86D2043A8652868036001932C
:1089AC0001250420384042424241029840072846A3
:1089BC0000D510466E0201280AD1082038404342E7
:1089CC00434102980007284600D5184600282FD1AD
:1089DC004B49886DC00602D4886D304388650B689E
:1089EC00D8680005800F1ED14548807E00281AD11A
:1089FC001868000717D59868400709D458680C21E7
:108A0C0088435860FF200230424C2168814307E0C4
:108A1C003B48846D20212143816504465C34C16D43
:108A2C000120084320603A48012101670C2018609E
:108A3C008023384618404442444102980006284698
:108A4C0000D52046002807D1012000042C4CA16D34
:108A5C000143A1652068036001231C0239462140B3
:108A6C00484248410299C905294600D501460029CA
:108A7C0006D15804224A916D014391651068046037
:108A8C00394631404842484102993142294600D08A
:108A9C000146002906D19804194A916D014391654C
:108AAC00106806601022394611404842484102992C
:108ABC00C906294600D50146002911D11048046881
:108ACC00006B002802D0E068800708D098020C4E9A
:108ADC00B16D0143B165F06D01990843F0652260F9
:108AEC00580307407A427A410299890401D403B0B1
:108AFC00F0BD1500FBD102490968086003B0F0BD58
:108B0C00640A00200024014071C0000814BE000853
:088B1C00E8090020BC0A00205A
:108B2400F0B581B06A4801F097FB6A486A4D29465E
:108B34005CC85CC15CC85CC15CC85CC15CC85CC12D
:108B4400482001262E5468206864286C401C286440
:108B5400624F7868002806D53846083860490160B5
:108B64006049016078687D20C1005F48426A5218FC
:108B740033043C681C4215D0446A944218D23C68C1
:108B84001C420FD0446A944212D23C681C4209D061
:108B9400446A94420CD23C681C4203D0446A944216
:108BA400E7D305E03A68514B5C1C3C601A4268D03C
:108BB4007968C90702D07968B14379603E2181643C
:108BC400067406756846FBF795F8002800D0FEE7A2
:108BD4000CCD474C2046083DFAF7D4FF0028FED1BF
:108BE400AA68EB6820460830FAF7CCFF0028FED1CB
:108BF4002A696B6920461030FAF7C4FF0028FED1B9
:108C0400AA69EB6920461830FAF7BCFF0028FED1A8
:108C14002A6A6B6A20462030FAF7B4FF0028FED196
:108C2400AA6AEB6A20462830FAF7ACFF0028FED186
:108C34002A6B6B6B20463030FAF7A4FF0028FED174
:108C4400AA6BEB6B20463830FAF79CFF0028FED164
:108C54002A6C6B6C20464030FAF794FF0028FED152
:108C6400AA6CEB6C20464830FAF78CFF0028FED142
:108C74002A6D6B6D50342046FAF784FF00281DD00E
:108C8400FEE7426A5118B2043B68134290D0436A2B
:108C94008B428DD23B6813428AD0436A8B4287D27F
:108CA4003B68134284D0436A8B4281D23B681342AF
:108CB40000D17DE7436A8B42E6D379E7F007796810
:108CC40001437960786800F015F801B0F0BDC04642
:108CD4007ABD000850B2000868000020102002404D
:108CE40023016745AB89EFCDE8090020FAC30000F2
:048CF40000F0010883
:108CF800F0B588B0A3490A78A34802704A78427050
:108D08008A788270CA78C2700A7902714A79427187
:108D18008A798271CA79C2710A7A02724A7A42726F
:108D28008A7A8272CA7AC2720A7B02734A7B427357
:108D38008A7B8273CA7BC2730A7C02744A7C42743F
:108D48008A7C8274CA7CC2740A7D02754A7D427527
:108D58008A7D8275CA7DC2750A7E02764A7E42760F
:108D68008A7E8276CA7EC2760A7F02774A7F4277F7
:108D78008A7F8277C97FC17784490A782023C254C1
:108D88004A782123C2548A782223C254CA782323DA
:108D9800C2540A792423C2544A792523C2548A79B1
:108DA8002623C254CA792723C2540A7A2823C254D4
:108DB8004A7A2923C2548A7A2A23C254CA7A2B238C
:108DC800C2540A7B2C23C2544A7B2D23C2548A7B6B
:108DD8002E23C254CA7B2F23C2540A7C3023C25488
:108DE8004A7C3123C2548A7C3223C254CA7C33233E
:108DF800C2540A7D3423C2544A7D3523C2548A7D25
:108E08003623C254CA7D3723C2540A7E3823C2543B
:108E18004A7E3923C2548A7E3A23C254CA7E3B23EF
:108E2800C2540A7F3C23C2544A7F3D23C2548A7FDE
:108E38003E23C254C97F3F228154554A11784023AA
:108E48000793C15451784123C15491784223069322
:108E5800C154D1784323C154117944230593C15493
:108E680051794523C154917946230493C154D1794A
:108E78004723C154117A48230393C154517A492393
:108E8800C154917A4A230293C154D17A4B23C154D5
:108E9800117B4C230193C154517B4D23C154917BC9
:108EA8004E230093C154D17B4F23C154117C5025CC
:108EB8004155517C5123C154917C52240155D17C98
:108EC8005323C154117D5423C154517D5527C15595
:108ED800977D56214754D27D5727C25507682D4A9A
:108EE800176187889782C788D78207891783478938
:108EF800178587895785C7899785078AD785478AB8
:108F08001786878A5786C78A9786078BD786478B9F
:108F18001787878B5787C78B9787078CD787478C87
:108F2800079E9753878C069E9753C78C059E975329
:108F3800078D049E9753478D039E9753878D029EF6
:108F48009753C78D019E9753078E009E9753468E61
:108F58005653858E1553C48ED452038F5352418F66
:108F68005823D152818F5A23D152C18F0A4B198469
:108F7800002902D05E2101235352C06C506008B012
:108F8800F0BDC04600F001086800002020F001088C
:0C8F980040F00108FC060020E809002061
:108FA400F0B583B00D460190914801F055F9914F09
:108FB40038697969904E03C6388B3080388D70805B
:108FC400788DB080B88DF080F88D3081388E7081C6
:108FD400788EB081B88EF081F88E3082388F7082AE
:108FE400788FB082B88FF082F88F30834020385A5F
:108FF40070834220385AB0834420385AF083462084
:10900400385A30844820395A71844A21795AB184B3
:109014004C21795AF1844E21795A31855021795A5B
:1090240071855221795AB1855421795AF185562195
:10903400795A31865821795A71865A21795AB186DA
:109044006E4C083E002D02D12146203101E0394604
:109054006431098801253554F18768207064306CC7
:10906400401C30640198002804D0654801F0F4F8ED
:109074007868F064634F7868002806D53846083865
:10908400614901606149016078687D20C000616ABE
:1090940009182A043B68134215D0636A8B4218D21C
:1090A4003B6813420FD0636A8B4212D23B6813426F
:1090B40009D0636A8B420CD23B68134203D0636AC3
:1090C4008B42E7D305E03968514A531C3B60114297
:1090D40068D07868C00702D07868A84378603E20DA
:1090E400A0642574257502A8FAF704FE002800D0B0
:1090F400FEE70CCE474C2046083EFAF743FD002815
:10910400FED1B268F36820460830FAF73BFD002828
:10911400FED13269736920461030FAF733FD002816
:10912400FED1B269F36920461830FAF72BFD002806
:10913400FED1326A736A20462030FAF723FD0028F4
:10914400FED1B26AF36A20462830FAF71BFD0028E4
:10915400FED1326B736B20463030FAF713FD0028D2
:10916400FED1B26BF36B20463830FAF70BFD0028C2
:10917400FED1326C736C20464030FAF703FD0028B0
:10918400FED1B26CF36C20464830FAF7FBFC0028A1
:10919400FED1326D736D50342046FAF7F3FC00288B
:1091A4001DD0FEE7616A0818A9043A680A4290D003
:1091B400626A82428DD23A680A428AD0626A8242E4
:1091C40087D23A680A4284D0626A824281D23A687B
:1091D4000A4200D17DE7626A8242E6D379E7E80772
:1091E4007968014379607868FFF784FD03B0F0BDC6
:1091F40090BD0008FC06002068000020E80900205B
:109204000AC100081020024023016745AB89EFCD55
:08921400FAC3000000F001089C
:10921C00F0B581B0544801F01BF8012529025348E0
:10922C00415A534E3184E021415AB184E221415AD2
:10923C007184E421415A3185E621415AF18421217E
:10924C00C900415AF18583214900415A3186412197
:10925C008900415A718581214900405AB085454F9A
:10926C007868002806D538460838434901604349D8
:10927C00016078687D20C1004148426A52182B0475
:10928C003C681C4215D0446A944218D23C681C427B
:10929C000FD0446A944212D23C681C4209D0446AF2
:1092AC0094420CD23C681C4203D0446A9442E7D3EB
:1092BC0005E03A68334B5C1C3C601A4230D079684C
:1092CC00C90702D07968A94379603F21816405748C
:1092DC0005756846FAF70AFD002804D02A4800F004
:1092EC00B7FF01B0F0BD326A736A284C2046FAF71A
:1092FC0045FC00280FD1B26AF36A20460830FAF711
:10930C003DFC002807D1326B736B10342046FAF702
:10931C0035FC002820D01E4800F09AFF01B0F0BDAB
:10932C00426A5118AA043B681342C8D0436A8B4264
:10933C00C5D23B681342C2D0436A8B42BFD23B6852
:10934C001342BCD0436A8B42B9D23B681342B6D0AD
:10935C00436A8B42E7D3B2E7E80779680143796047
:10936C00786801B0F0BDC046E8C30008FC060020D8
:10937C00000000201020024023016745AB89EFCD8F
:10938C00E8090020FAC3000017C1000800F8010822
:04939C00A6BD000862
:1093A000F0B58DB00246084665384442444108464F
:1093B0006F3843424341234303D102206F2903D135
:1093C00004E001206F2901D0652901D10A3000E0B5
:1093D00009309A4D6A609A4E35600127BA023C0303
:1093E00065290492059406D06F2902D103214A020F
:1093F00001E000221446AC602A610021002B00D15C
:109400007903E96000F080FC8E4B002202F090F8B6
:1094100000F032FC2A688C498A42069009DD8B49AB
:109420008A420CD08A498A4209D08A498A4206D0A7
:1094300046E089498A4202D088498A4240D1842440
:109440002859002846D1802000262E5428688149BA
:10945000884233D1B8038449CA680243CA60CA68E3
:109460000240089208980868384308600868384045
:1094700007900C970B960A960220039009900920FA
:1094800040020890079805200007029008A9019162
:10949000FAF714FD0C970B960A9703980990049815
:1094A000089002980199FAF709FDFF2000066F491C
:1094B0000A6882430A60F8066D490860604E09E058
:1094C0003A0249326648674900F0C8FE84242859A8
:1094D0000028B8D02420285128680168B9430160C9
:1094E000FBF786F8012827D0A86A002801D0FBF7EF
:1094F000FBFAB903286882680A438260F90382682C
:109500008A43826001685B4A0A400260F90542684A
:109510000A434260B90602680A430260FF2421063A
:1095200042690A4006990A43426101683943016071
:10953000FBF7D6FB002801D072B6FEE731680A4679
:1095400080329068202809D18B680598834202D127
:109550000869002802D01078012803D14C4800F097
:109560007DFEFEE70D465C3500200690C86617704C
:109570002C806C8027368E65002B0AD03E07B342C4
:109580000BD03E03B3420DD10E69002E0DD13A4CE3
:109590000BE00E69002E07D107E00C69002C03D008
:1095A0003F2402E0A88001E07F24AC80D060222428
:1095B00094600E68B4683C43B460380204907C0741
:1095C000486EA04202D1A889FF280DD90598834290
:1095D00002D1086900282DD02B4B069C049D1470E5
:1095E0000B672035334610E00598834202D10869A5
:1095F000002821D0224D069C3346083314700D6795
:1096000030680499084330603D070D4A2620145401
:109610004720C0001F4911508D2080001B49115068
:109620001868284318609484D46114841C3294719F
:109630000DB0F0BD134BD0E7104DDCE7DC08002087
:10964000C004002000000C40FF4B0040004C0040D4
:1096500000800040003801400044004000480040C5
:1096600071C0000897C100083410024018E400E0FF
:1096700000E100E0FFFF00FCFF010000A94F00082F
:109680006D4E00088BB4000821B40008700B002058
:08969000C8BD0008060A002015
:10969800F0B58AB098480168CC69086809904868AC
:1096A800012007900007069088680890230753D088
:1096B8000698401C089A104001252A0216462036B2
:1096C800099F3E40064347D03A4056425641E2077A
:1096D800079A00D03246002A05D10D628C22864FA7
:1096E800BE582E43BE50089A15406A426A41A607E2
:1096F800079E00D51646002E08D102220A628C2247
:109708007D4EB658042737437B4EB7506A426A41AC
:109718006507079D04D4002D04D0002B0CD41BE052
:109728001500FAD104220A628C22734FBD58022612
:109738002E43BE50002B0FD5421E9041099A920627
:10974800079A00D40246012A06D1082008628C2212
:10975800694DAB580343AB500125E805049020053B
:1097680013D50898049A1040AA06099B1A401018A5
:109778000BD0E8020862882020225F4B1A50842010
:109788001A505E4805755E4A855403952020274681
:10979800059007401ED00898069A1040099A059B24
:1097A8001A40024316D04520C000544A1358882551
:1097B800514E7559222D00D094E0FE2B00D991E02E
:1097C800D3184D6A27269D554D4B039DD5541358E4
:1097D8005B1C1350802326461E402ED00898049AFE
:1097E8001040099A1A40024327D04448006884224E
:1097F8008258212A14D1024656321588002D0FD0DE
:1098080005680195056D02952D780092019A95627B
:10981800029A551C0565009A1088401E108007E0C2
:10982800006802689A430260026840251543056093
:10983800324D23200001039A2A5402934025099AA5
:109848002A4050425041620600D5079007980028E8
:109858000DD10868A84308608420274B059A1A5040
:10986800284800220270882022241C505A678C2223
:109878002148805800282AD0882422201E4B1851BD
:10988800002F09D0089B079106991940099F059B4D
:109898001F400F4307991CD1002E18D0089B049A2B
:1098A8001340099A029E32401A4310D00A68AA430C
:1098B8000A608421104B059A5A50185126200F49E6
:1098C80000220A5423200001039C0C545A670AB052
:1098D800F0BD8869082303438B610020064988503E
:1098E8000AB0F0BD8869082202438A6180232646AF
:1098F8001E40A2D072E7C046DC080020C004002049
:0899080031020000E60400201A
:109910000122D20703004B403AD430B4431A01D29B
:10992000C01AC9184B004400240EFF2C29D0002C6B
:1099300024D01B0E20D0E31A182B1DDC0902114382
:10994000C40D000210435D4219350A00AA40D20935
:10995000D940451801D36D080234013CE405280ABA
:109960000121C9072D062A438A4160414100090EA1
:10997000FF2901D3C00DC00530BC7047C00FC00720
:10998000FAE74202F8D07F2000010C300005F3E72F
:10999000A4465140431A02D25340C01AC9184B0082
:1099A000090211431B0E4400240EFF2C41D0002B52
:1099B00010D05B421B19012B10D322D1C30D4002E2
:1099C000401A10D3DB050100400AC90591415841F6
:1099D000644670472442FBD10020F9E7C30D4002E2
:1099E0004900401AF4D0002101314000FCD38C42E0
:1099F00004D95B1ADB05400AC018E9E7180AC0075A
:109A0000E6E7192BE4D801330C00D940DC414C4087
:109A1000012C4941C30D00021043441A01D4A40093
:109A20006408013BDB05200A240694415841644642
:109A30007047FF2B01D04102CAD07F2000010C30BB
:049A40000005C5E771
:109A44000122D2075140014B184700001599000824
:109A540030B405004D400124E407254042004B008A
:109A6400120E32D01B0E3CD0FF2A33D0FF2B3FD036
:109A7400D21800022043000A09022143090AC4B291
:109A84004C43000AC3B24B43000A4843210A5B1803
:109A9400190A091801D44900013A080A7F3A2ADB55
:109AA400FE2A0FD2D2051C43240601D001242143EF
:109AB400C9B280295041802901D14008400028437F
:109AC40030BC7047FF20C005F9E71B0EFF2B0AD0FE
:109AD4002800F5E7400206D1FF2BF3D1490202D159
:109AE400F0E7FF2AF4D17F2000010C300005E7E7FE
:109AF4004902F8D1E6E743020132E9D15B120233AD
:089B0400E6D9D805E4E7C046EC
:109B0C0030B405004D400124E407254042004B00D1
:109B1C00120E26D01B0E34D0FF2A2DD0FF2B35D0A1
:109B2C00D21A000220430902214343084908A00D20
:109B3C005B1A02D2013A5B005B185B008B4200D3CC
:109B4C005B1A4041F9D37F3222DDFF2A06D2D205BF
:109B5C00C91A8B425041284330BC7047FF20C005C6
:109B6C00F9E71B0E03D0FF2B12D1490210D07F2036
:109B7C0000010C300005EFE74002F8D1FF2BEDD1CE
:109B8C00F5E7FF2AEAD14002F1D1E7E74902EED12D
:049B9C002800E1E7D5
:109BA00002000A43520008D0884204D1400001213B
:109BB0000906C84201D90020704701207047C046FD
:109BC000012212064300DA4211D84B00DA420ED8C5
:109BD00002000A43520008D003D28842804101307B
:109BE000704781428041013070470120704700205A
:049BF0007047C046B4
:109BF400012212064300DA420FD84B00DA420CD895
:109C040002000A43520008D003D2814280414042FC
:109C14007047884280414042704700207047C046E8
:109C2400012212064300DA420FD84B00DA420CD864
:109C340002000A43520008D003D2884280414042C5
:109C44007047814280414042704700207047C046BF
:109C540041000DD2090E7F390AD449421F3105D47F
:109C640000020122D2071043C8407047C81770474A
:049C74000020704715
:109C78004A0010D2520D03231B02FF33D21A0AD412
:109C880052421F3209D4400DC90208430123DB07A1
:109C98001843D040704700207047D0177047C0461F
:109CA800420017D2120E7F3A14D480231B06202AB2
:109CB80006DA52421F3200021843D0400021704792
:109CC80052423F3209DB010219430800D041D1401A
:109CD80048407047002001007047D01701007047C6
:109CE8009D2201000AD002D4013A4900FCD5D205D0
:109CF800080A0906494100D3012950417047C04666
:109D080042221201033A010007D002D4013A001896
:0C9D1800FCD51205C30A400599187047DD
:109D2400BD22094210D003D4013A00184941FBD5A1
:109D3400D2050128804101300143080A090649413E
:109D440000D301295041704700490847E99C0008A5
:109D54004B1801225205DA4217D25B0D0722D201B9
:109D64009B1A0FD9FF2B13D2DB05CA0FD20713435B
:109D74000903020D1143490AC200524100D90131BD
:109D8400C8187047C80FC007704706D1002804D10F
:109D9400C80F0002FF30C00570470123DB070A002B
:109DA400C900400F084398431A4010435B0A184304
:049DB4007047C046EE
:109DB800F0B581B00A464149C30D5C1EFD2C58D848
:109DC800FD24E443D50DFF3DA54252D306460E407F
:109DD800491C0140964260D90091DCB20123DD059F
:109DE800002C03D0691E0840284309E0AE4206D281
:109DF8009F05641E7000BE420646FAD300E0304656
:109E0800D10DCEB2002E03D0691E0A402A4308E0C5
:109E1800AA4206D29F051146761E4A00B94211464B
:109E2800FAD3B4420ADD811A02D4904201D109E082
:109E38000146641E4800B442F5DC3446861A03D451
:109E4800904202D1009A11E00646AE4206D2990528
:109E5800641E70008E420646FAD300E03046002C9D
:109E68001FDD611E009A8018C9054218104601B00E
:109E7800F0BD4500124CA5421BD25500AC42F5D9A5
:109E880006460E40FF24E5050E4CAE4213D0002EC8
:109E98000BD10A420246E9D10DE000D001460A463C
:109EA800E4E7191BC8400021DCE70A4003D0AA42B6
:109EB8008ED10246DAE72246D8E7C046FFFFFF7F89
:089EC800010000FF0000C07F53
:109ED000C10DC9B24A1EFE2A19D27E2903D8002814
:109EE00013DA104870479529FCD87F390C4A0A418B
:109EF0000240134603D5094B5B1CCB40D318884066
:109F0000400200D01A4610467047002070470029D2
:109F1000E8D10121C90708407047C046FFFF7F0014
:089F2000000080FF000080BF7B
:109F280030B5514343435C18010C130C0D005D43DD
:109F3800641992B2514380B242430D0C090452187D
:109F480065415843010C00048018694130BDC04682
:109F5800CA1751408B1A17D0C1174A409446484037
:109F6800411A48081A0000E052008242FCD9002039
:109F780000E05208914200D3891A40419A42F8D130
:109F880062465040801A704710B500F07DF810BD49
:109F980007B5FFF7DDFF0EBC4243891A00BDC04676
:109FA8000A0015D00300400800E052008242FCD9A4
:109FB800002000E052089B1A06D340418A42F9D19A
:109FC800704752089B18F8D200188A42F9D1704796
:089FD80010B500F059F810BDAE
:109FE00038B504004D42FFF7DFFF4543611938BD26
:109FF000002B09D1002907D110B51100FFF7F0FFA0
:10A000000A000021002310BD70B400240125ED07D3
:10A01000002B07D1002905D0834203D21300002270
:10A020002C0000250026A419994200D1904212D993
:10A0300092185B4103D2EE076D086408F3E7DE0770
:10A040005B08520892190126F6079B1903E0DE0708
:10A050005B0852089219801A994103D364416D41FB
:10A06000F5D30FE024196D410AD2DE075B085208D0
:10A07000921980185941F5D364416D41E7D301E04D
:10A080008018594102000B002000290070BC704765
:08A09000002000217047C046CA
:10A0980003490868002800D07047024808607047E4
:08A0A800400B0020480B0020D2
:10A0B0007F2805D8034A125C0348405C1040704773
:0CA0C0000020704768C4000839C2000886
:10A0CC007F2805D8034A125C0348405C1040704757
:0CA0DC000020704768C4000839C200086A
:10A0E800411C02780130002AFBD1401A7047C04653
:10A0F800002A03D0013A8B5C8354FBD17047C046D9
:10A1080000220B0011001A00002A02D0013A8154E3
:04A11800FCD17047BF
:10A11C00F0B581B00022002933D00378002B30D069
:10A12C00032302469A4316680024E5438707FF0E73
:10A13C00BD40ED43354306461E407118042900937B
:10A14C000AD3124EAF19104BAB433B4204D1091F3B
:10A15C005568121D0329F5D82B060DD02B041B0EA8
:10A16C0007D02B021B0E06D02B0E009C04D004240F
:10A17C0002E0012400E002248C4200D30C46101AA9
:10A18C000219104601B0F0BD80808080FFFEFEFEFB
:10A19C00F0B581B004467F20C605002C00960FD088
:10A1AC00E11722464A40571AC6050A4DF80704D053
:10A1BC0029683046FFF748FC06462D1D7F08F5D16F
:10A1CC0000983146FFF79CFC002C00D4304601B0BF
:08A1DC00F0BDC04624B30008E9
:10A1E400F0B503AF93B06E46F51D2135F41D393437
:10A1F40074613362F261F160306100F0FDFEB060C1
:10A20400C21D07218A436946B1616946881A706094
:10A214008546F41D1D34002124222046FFF776FFD5
:10A224000B487169F2680A6048600A48286030691E
:10A234002862B06868617068E8602046F169326A33
:10A2440000F01EF8B1698D46FC1F053CA546F0BD23
:08A2540003B90008FFFFFF7FC2
:10A25C0083B010B581B0044603A80EC00548006851
:10A26C0003AA0092214601F073FA01B010BC02BCA3
:08A27C0003B00847640B002049
:10A28400F0B59FB014460F460021159001600120DF
:10A2940002020C92460282020392C202029203223A
:10A2A4000A929202059202031792420307928203D2
:10A2B40004920090C00316900891C84301900F9631
:10A2C4003978252908D0002901D100F060FE7F1CCF
:10A2D400159801F0E4F9F3E7FF1C089BB81E057814
:10A2E4002A46203A102A2BD880219200184602A32D
:10A2F4009A5803469746C04641A3000861A3000844
:10A3040061A300085BA3000861A3000861A300081F
:10A3140061A300084DA3000861A3000861A300081D
:10A324008BA3000851A3000861A3000855A30008EB
:10A3340061A3000861A3000859A3000840210AE0B2
:10A344005E2D179907D009E0169904E0202102E058
:10A35400102100E031460B437F1CBFE77F1E2946D6
:10A364003039C9B20929139419D800240A21614348
:10A374006C18303C791C3D782A46303AD2B20A2A0D
:10A384000F46F3D30CE001CC0028139401D510211F
:10A394000B43C1174840441A781E057800E0002496
:10A3A40000202E2D08D13D782A2D07D17D78BF1CA1
:10A3B400139901C9139113E00E9018E07F1C2946EC
:10A3C4003039C9B209290FD80A21414368183038F5
:10A3D400791C3D782A46303AD2B20A2A0F46F3D382
:10A3E40000280E9001D502E00E900C980343184605
:10A3F400E1172A46683AD301D2B252089A18D2B267
:10A40400092A2BD8920002A39A5803469746C046BD
:10A414003DA4000847A4000851A4000871A4000842
:10A4240071A4000871A400084BA4000871A40008DA
:10A4340071A400084BA400083D78682D10D10820B1
:10A4440008E0022003433D787F1C0FE03D786C2D2B
:10A4540009D1022003437D78BF1C07E0034605E0D1
:10A464007F1C042201E07F1C012213438C43462DF0
:10A474000B941BDD2946633915292BD8139CC04640
:10A484007944097949008F44460B421CC30A0B0ADC
:10A494000A0A0A5966730A0A810A830A0A2E0FE70E
:10A4A400049803430021099119467AE0442D159834
:10A4B400139C08DD452D28D0462D00D000E70798D1
:10A4C4000343029824E0252D00D080E2252101F0E9
:10A4D400E6F8F5E6472D139C00D197E0582D00D0FF
:10A4E400EEE607980343CE4A782D00D120321906B0
:10A4F400C81709900C98034201D0CA480340194672
:10A504000498099B134009934BE00798034303986D
:10A514000343059A7EE0264624780B98421E159D37
:10A52400284619461292149301F00BF92846214645
:10A5340034460F9E01F0B3F8241DDFE0180700D560
:10A5440049E29807159801682068016000D446E242
:10A554000021416043E20C980342194601D0B148FE
:10A5640001401A06D217302010400990049818E0D0
:10A57400069718060C990B43C01723210140099133
:10A5840004CC1394002708200E90B2E101CC8DE096
:10A594000C98034201D0A3480340194604980022B2
:10A5A400099202220A400142069706D1002A09D1E3
:10A5B400231D002722461C460AE0002A12D104CC9F
:10A5C400D01715E0E21D07239A4357681446083450
:10A5D40013684A0714D408220A4000D0DBB2002AC8
:10A5E4000FD1FCE0E41D072294432268606808341C
:10A5F4004B0708D40B0700D5DDE013460746DDE022
:10A604009BB20027EBE013B21204D6E00798034391
:10A61400059A13430C98034201D00E9800E00620DB
:10A6240014931340991A4A424A410E92002800D0CA
:10A634000E90E41D0720844303CC083CFFF788FBFD
:10A644002546044601F024F80835139500282046D1
:10A654000ED00021FFF7E4FA149B1A4607990A402A
:10A66400002813D0002A704800D070482C461BE004
:10A6740001F005F8002846D00798149B03426C4863
:10A6840000D06C486C490B402C460FE0002A6B4903
:10A6940000D06B49002A01D0694800E067482C4685
:10A6A400401C9A0600D5084663490B400028654EB5
:10A6B40000D0064619465B48014014910C980342A9
:10A6C4001394304602D1FFF70DFD02E00E99FFF717
:10A6D40023FD05460B98441B15981499224601F056
:10A6E40030F8002D129407D0159C3178204600F0E4
:10A6F400D6FF761C6D1EF8D1139C0F9E1498C006CD
:10A7040000D4DDE55DE10126204601F080F8054630
:10A71400002801D0F007444012961EA9204601F0FB
:10A7240094F81E980A9948430A21FFF713FC064639
:10A734001E90002D03D0602014990143149100252C
:10A7440020462946FFF72AFA002818D1701CFFF783
:10A7540023FD01462046FFF74BFA00281E9806D039
:10A76400411C1E91801CF2E71E98401E1E90FFF7AC
:10A7740013FD01462046FFF753FA0028F4D1149A3A
:10A7840016460598064012998B029E4200D128E194
:10A79400864209D11E980E99814200DC22E10421EF
:10A7A400C943884200DC1DE112930398024200D0A1
:10A7B40020E10E9D06E253B21206D717002F05D4EE
:10A7C4008A060AD44A060AD5202007E000225B4202
:10A7D400BA412D200990174601E02B2009901A4612
:10A7E4000C98014201D00F4801400B460C980142DD
:10A7F400139401D00E9800E0012000246E2D0E90D9
:10A8040039DD6F3D092D00D994E0C0467D442D7992
:10A814006D00AF44196E8F8F8F8F368F8F6EC04649
:10A8240058300000FFFDFFFF4BC2000846C200087D
:10A834000CC5000808C50008FFFEFFFF55C200084C
:10A8440050C2000893BA00081046384372D0D008AA
:10A8540079074018014607201040303018AA1055D7
:10A86400C808FF087A0780180A463A43641C002A7D
:10A874000A46EFD15EE0582D3BD0642D01D0692DFE
:10A8840058D11046384355D01946169801400D91B9
:10A894000021149314463B460D9800280F4608D017
:10A8A40008460A990840032803D118A82C21C15549
:10A8B4007F1C0A2200252046194612932B46FFF7D7
:10A8C40095FB1094044611910A222B46FFF72AFBAC
:10A8D400109A101A3021014318A8C155791C092077
:10A8E400801A12988541119F0F9E149BD3D30C4656
:10A8F40020E0104638431CD007981D460342FA480E
:10A9040000D0FA48134611093A07891800240A4668
:10A914000F211940415C18AB195511093F093B0738
:10A92400C91813463B43641C002B1346EFD12B4636
:10A9340000E00024099A511E104688410B99091B16
:10A94400FF2A00D9491E069F081A0E990D1BE91704
:10A954008D43421B3342149305D11598194600F0D8
:10A96400F0FE149B0022099E310A129204D015981D
:10A9740000F095FE129A149B002E3146159E04D0C9
:10A98400304600F08CFE129A149B3046194600F0B3
:10A99400D8FE302130462A4600F0A3FF012C0ADB02
:10A9A400641C18A80019801E0178304600F077FE58
:10A9B400641E012CF5D81498C006139C0F9E00D475
:10A9C4007EE420211598129A00F08BFF78E4002D84
:10A9D40000D075E4EBE22068159909680170241D24
:10A9E4006EE41E98119626282ED12046CC49FFF7F6
:10A9F4008BF82FE01E980E2800DDE3E0C0430E998B
:10AA04000E18102E00DB1026100600D5D9E0002EFB
:10AA1400354600D1D6E03046FFF7BEFB2146FFF7AE
:10AA240017F83F210906FEF771FFFFF74FFABD49FA
:10AA3400FFF7C0F900252946FFF7B0F8002800D138
:10AA4400BFE0761EE7D1BDE04042FFF7A5FB2146FB
:10AA5400FEF7FEFF064600252946FFF79FF800286B
:10AA6400139C15D1304600F013FE0028304611D057
:10AA74000021FFF7D5F8149B1A4607990A400028CD
:10AA840000D196E0002AA84800D10DE6A7480BE6BD
:10AA9400099527E00995A34C2146FFF78FF81E9DE1
:10AAA40000280BD030462146FFF72EF806462146F3
:10AAB400FFF784F86D1C0028F4D11E957F20C4058F
:10AAC40030462146FFF7ACF800280BD030469549B4
:10AAD400FEF7BEFF06462146FFF7A2F86D1E0028CA
:10AAE400F4D11E950598119981420E9801D005461E
:10AAF40000E0451E8B4C0028294600D1002111910D
:10AB04004842FFF749FB019900F083FE3146FEF706
:10AB1400FDFE06462146FFF751F8002807D01E988F
:10AB2400401C1E9030462146FEF7EEFF0646149A5E
:10AB340011980D96002839D0119502990B4680334F
:10AB440013408B4200D0ABE0102800DB10200546F8
:10AB5400FFF722FB3146FEF77BFFFFF7A3F81090C7
:10AB640008430998119000D19AE00A220023109812
:10AB74000E46FFF73BFA002D00D190E01A4300D0B7
:10AB84008DE0119531460A2200231098FFF72EFA22
:10AB940010900C460A220023FFF728FA1198401E51
:10ABA40011907DD01A432146EDD079E00998119097
:10ABB40076E0002A5E4900D05E49002A6DD05D48E7
:10ABC4006EE535461E9810386942884200DC084616
:10ABD400FFF7E2FA019900F01CFE2146FEF796FE0B
:10ABE40004461E98401CFFF7D7FA01462046FEF79C
:10ABF400FFFF1E99002800D0491C149800291195C4
:10AC040011D4112914D3084610381E901020401A6C
:10AC1400FFF7C2FA2146FEF71BFFFFF743F806468B
:10AC24000C46002012E00D9400261E9634460FE0D8
:10AC340000201E902046FFF735F8254606460C46B0
:10AC4400FFF76EF801462846FEF7FAFE0D901498B9
:10AC540012998843DB49083100250A4608326D1CE5
:10AC64000B684968F31A23468B411146F6D21095B6
:10AC7400119B002B0099149A01D1D1B2C909520633
:10AC8400920F01D1494200E0C9431E9A891A0B9AD6
:10AC9400D21A5118491B024676E0C74800E51195BF
:10ACA400119D002D0098149A01D1D0B2C0090B99BE
:10ACB400491B081A411F1E9C17980242129E01D17B
:10ACC40010963FE00E91032120461091FFF762F9A0
:10ACD400881C042822D8C046784400794000874460
:10ACE40007132B071300C046F8C40008E8C4000883
:10ACF400641E1E940D98B149FEF7AAFE0D900E999C
:10AD0400491E022010901AE0A41E1E940D98AC490E
:10AD1400FEF79EFE0D900E99891E10E000200CE0B7
:10AD24009976967E000020414BC2000846C2000876
:10AD340055C2000850C20008012010900E99149AC0
:10AD4400E81785435006800F119500D0491E0E91D7
:10AD5400F502204600F08BFD632802DD0E98401EAC
:10AD64000E9014980D9CA84314902046FEF79AFF69
:10AD7400254606460C46FEF7D3FF01462846FEF755
:10AD84005FFE149A0D900E99C8170D4685430F98CF
:10AD940010300242149208D1012906DB20211598B3
:10ADA40000F07DFC6D1EF9D1149A402010409106EC
:10ADB40003D400280AD0202104E0002801D02D214A
:10ADC40000E02B21159800F06AFC149AD0060AD4EE
:10ADD400002D08D03021159800F061FC6D1EF9D1CA
:10ADE40000200E9000E00E951099491E0D46C800F3
:10ADF400744A111849681258B01A2046884101D281
:10AE0400302007E03020B61A8C41401CB31A234688
:10AE14008B41F8D2C1B2159800F041FC2946002DAF
:10AE24001498E2D10146029801401291159E0BD06C
:10AE34001E98012808DB401E1E903021304600F089
:10AE44002EFC1E980028F6DC802014990840119CE2
:10AE540020430E9D4BD02E21304600F020FC102CB8
:10AE6400264600DB1026F017344684431298002847
:10AE740001D1204601E01E98201AFFF78DF9014602
:10AE840011981094001B0B90012E23DB0D98FEF7F4
:10AE9400DFFDFEF707FF04460E46109B5B1ED8003D
:10AEA400484A111849681258A01A3046884112932A
:10AEB40001D2302007E03020A41A8E41401CA31A8E
:10AEC40033468B41F8D2C1B2159800F0E8FB129BCF
:10AED400002BE3D10B980028159E119807D01099E8
:10AEE4000C1A3021304600F0DAFB641CF9D30398C5
:10AEF400149901423BD00798014201D0452100E05A
:10AF04006521159C204600F0CAFB1E9800282046A7
:10AF140004D42B2100F0C3FB1E9805E02D2100F082
:10AF2400BEFB1E9840421E9064280FDB6421FFF78D
:10AF340039F801463031159E304600F0B0FB1E98BA
:10AF44006421FFF727F808461E9100E026460A21EF
:10AF5400FFF700F801463031304600F0A0FB1E98A0
:10AF64000A21FFF717F83031304600F098FB002D26
:10AF7400139C0F9E01D1FFF7A3F9159C20212046B5
:10AF840000F08DFB6D1EF9D1139CFFF799F9159C08
:10AF9400E068002805D006CC083C914201D2089A0A
:10AFA4004254204600F0C0FB20681FB0F0BD00F002
:10AFB400BBFB0198F9E7C04655C2000800002041D8
:08AFC4000000C842C030000883
:10AFCC00084B1B6883420AD0074B1B68834206D090
:10AFDC00064B1B68181A431E9841404270470020CC
:10AFEC00FCE7C046680B0020640B00206C0B0020B3
:04AFFC00402070473A
:0CB0000010B5006800F0C8F810BDC04694
:10B00C0003230F480F4A036143610F4B8261C361F5
:10B01C008023DB000362002383624362C362026607
:10B02C000A4A426610228266094A0367C36643676E
:10B03C001178013AC1540133102BF9D17047C04635
:10B04C003408002054B30008C0000020240B00205A
:04B05C0083B30008B2
:10B06000F8B54746CE46C5688368040040689946EF
:10B070005B1B80B50E00170098464019934207D914
:10B08000FFF73AF8ED19E560C0BCB946B046F8BD27
:10B090001A00FFF731F84B463100ED19ED1A2A007E
:0CB0A00060684144FFF728F8EDE7C04667
:10B0AC00F8B54746CE46002380B588460700160003
:10B0BC009946C56884681BE0013B5B1B641BB4426A
:10B0CC0000D934009C4200D91C007868220041460B
:10B0DC004019FFF70BF82D19A144A044361BBC688E
:10B0EC00631B5A1E93415B421D40FD60002E06D02F
:10B0FC003B699D42E0D3013B1B195B1BDEE74846D5
:08B10C00C0BCB946B046F8BD15
:10B1140070B50600431C5C00E4181D4BE400E01805
:10B124007400A419E4001B19DC6A1500012C06D074
:10B13400022C1FD0002C10D00024200070BD9A6A6D
:10B144005C6AA2421FD9013A121B2C00954200D915
:10B1540014002200FFF782FFEFE79A6A5E6AB242A8
:10B164000CD9013A961BB542E7D82A00FFF776FFBF
:10B174002C00E2E7FFF798FF0400DEE71B6AD21811
:10B18400013A961BEFE71B6AD218013A121BDCE75F
:04B19400340800205B
:10B19800F8B50B4B04001B780D001600002B0CD0E3
:10B1A800EFF31087012181F3108832002900200075
:10B1B800FFF7ACFF87F31088F8BDFFF723FFEFE731
:04B1C8003408002027
:10B1CC00072904D9024B41601860002303607047C3
:04B1DC00440B002000
:10B1E000000000000000000000000000000000005F
:10B1F000000000000000000000000000000000004F
:10B200000100000002000000030000000400000034
:10B210000600000007000000080000000900000010
:10B22000000000000000000000000000000000001E
:10B230000100000002000000030000000400000004
:10B2400000000000040000000200000008000000F0
:10B25000004B0000650001000100740EF00A420E70
:10B26000100E540B800CC409280AF401C2013200EC
:10B2700046006AFF9CFF5802100EFA000000000012
:10B2800000000000000000000000000000000000BE
:10B29000DB090020DC090020DD090020DE09002098
:0CB2A000D6BD0008CCB20008ACB200081B
:10B2AC00B1A00008B7B80008C3B80008CDA00008CA
:10B2BC00CFB80008DBB80008A7B800087BB80008B6
:10B2CC00D8BD000826C2000826C2000826C2000805
:10B2DC0026C2000826C2000826C2000826C20008A2
:10B2EC0026C2000826C20008FFFFFFFFFFFFFFFF7A
:10B2FC00FFFFFFFFFFFF0000DABD0008D8C1000808
:10B30C0026BA0008F5C100087DBA000827C200085B
:08B31C0030C2000884BA0008E9
:10B32400000020410000C84200401C4620BCBE4C26
:08B33400CA1B0E5AAEC59D7440
:10B33C0003480449091A08B5FFF742FF0CBC18472B
:08B34C00100C0020101000207D
:09B354005465726D696E616C00B4
:10B35D00455845433A20466163746F7279205265B2
:07B36D0073746F72650A00A2
:10B3740000000000000054545220524547474553F2
:01B3840000C8
:0FB38500455845433A20524553544152540A000B
:02B39400FEE7D2
:02B39600FEE7D0
:02B39800FEE7CE
:02B39A00FEE7CC
:02B39C00FEE7CA
:02B39E00FEE7C8
:02B3A000FEE7C6
:02B3A200FEE7C4
:02B3A400FEE7C2
:02B3A600FEE7C0
:02B3A800FEE7BE
:02B3AA00FEE7BC
:02B3AC00FEE7BA
:02B3AE00FEE7B8
:02B3B000FEE7B6
:02B3B200FEE7B4
:02B3B400FEE7B2
:02B3B600FEE7B0
:02B3B800FEE7AE
:02B3BA00FEE7AC
:02B3BC00FEE7AA
:02B3BE00FEE7A8
:02B3C000FEE7A6
:02B3C200FEE7A4
:02B3C400FEE7A2
:02B3C600FEE7A0
:02B3C800FEE79E
:02B3CA00FEE79C
:02B3CC007047C8
:10B3CE0030B584214158212918D102465632938A2C
:10B3DE00002B13D0016802E05B1E1C040ED01488F3
:10B3EE00002C0CD0CC692406F6D5046D25788D6220
:10B3FE00641C04651488641E1480EDE730BD0120C2
:10B40E00C0058A6882438A600868402202430A6047
:02B41E0030BD3F
:10B4200010B5882141582229016810D102465E32A8
:10B430005388496A1940836D19701188491E11801B
:10B44000816D491C81651188002905D010BD88696E
:10B45000082202438A6110BD0246883209214B014D
:10B4600001680C689C430C608B680124A3438B60CB
:10B470002023136000220267C36E012B03D10B68E7
:0AB480001024A3430B60C26610BD48
:10B48A0010B588214158222901680FD102465E323F
:10B49A0053884C6A1C40836D1C801488641E148077
:10B4AA009B1C83651288002A05D010BD8869082272
:10B4BA0002438A6110BD0246883209235B010C6887
:10B4CA009C430C608B680124A3438B602023136088
:10B4DA0000220267C36E012B03D10B681024A34319
:06B4EA000B60C26610BDFC
:02B4F000FEE775
:02B4F200FEE773
:02B4F40070479F
:02B4F60070479D
:10B4F80008D1002806D1F54204D801D3002A01D189
:10B508006D0D09D10020C143090DC904F0BDF9D161
:10B518001242F7D1640DF5D00020C143490549080E
:10B52800A6E000206146F0BDF0B50127FF070E0038
:10B538005E403E40B446BE0A4C18DD18F442D7D2ED
:10B54800F542E4D2640DECD06D0DEAD06419C9025D
:10B558003943460DC0023143DB023B43DB0A10B4DA
:10B568008E4685B297B26F43140C6C433E0CA419F7
:10B57800260C2404BFB227439CB26C43A419190CAF
:10B588006943250CA4B249190D04090C6419000C6F
:10B5980095B245433E0C76193743BFB2360C150CAD
:10B5A8004543AD19A6B2240CAD192E0437432E0C11
:10B5B80036199DB24543AD19ACB22E0C89191D0C34
:10B5C80045436D182E04290C3443704680B295B259
:10B5D80045433E0C76193743BFB2360C150C45432C
:10B5E800AD19A6B2AD19240C2E0437432E0C36190A
:10B5F8009DB24543AD19ACB22E0C89191D0C4543BB
:10B608006D182E043443290C75462D0C90B26843EE
:10B618003E0C80190604BFB23E43070CA0B23F1887
:10B62800120C6A43D019020C80B2240CA4189AB2E6
:10B638006A43121914042043120C89181B0C6B431B
:10B64800C91810BC01273D05294203D1B61940414C
:10B658004941013CFF077D0D013D641B0BDB6D007B
:10B66800AC4209DA240500254208BE41684161411F
:0AB6780066463143F0BD54E74EE78B
:10B68200FF2109064000884201D8002070470120AE
:02B692007047FF
:0EB69400012109064000411848424841704714
:10B6A20030B581B0044668460170206900280FD089
:10B6B2000CCC083C9A4233D26269531C63618154B8
:10B6C200A069616981422BD1204600F02EF827E063
:10B6D200E068002809D00CCC083C9A4220D2551CC4
:10B6E2009D4200D1002181541AE0A068002808D0B0
:10B6F2000CCC083C9A4213D2551C9D420DD0C9B2C3
:10B702000CE0236A002B0BD003CC083C884207D202
:10B71200694601222046984702E0002192008150AA
:0AB722002068401C206001B030BD1B
:10B72C0010B54269002A07D00446036A002B01D0E9
:0AB73C00216998470020606110BDEC
:10B7460080B5CB0606D4890501D5302100E020213D
:06B7560000F0C6F880BD02
:10B75C0070B514460D460646FEF798FC0146304679
:0AB76C002A462346FEF738FD70BDA3
:08B77600F7F7FDFCF7F7F1FC09
:10B77E00806A816D40220A438265C16D04220A43AC
:04B78E00C2657047D9
:10B7920010B58421415821290DD1014656310A881C
:10B7A200002A09D00268036D1C7894625A1C026553
:10B7B2000888401E088010BD0068016880229143FD
:0CB7C2000160016840220A43026010BDD3
:08B7CE0080B5FDF762FF80BDAC
:08B7D60080B5FDF75EFF80BDA8
:10B7DE00F0B581B01E4615460C4607461846FFF7D3
:10B7EE00EEFB0146002000290AD46543A54207D38B
:10B7FE00304639462A46FFF7FCFB2146FEF7CDFBC5
:04B80E0001B0F0BDD8
:04B81200C00F7047AC
:10B8160010B5FD22D343C20DD2B21446FF3C9C4262
:10B8260008D351184A1EFD2A05D8FF22D205904397
:10B83600C905084310BD0122D20710400129F9DBD2
:08B84600FF21C905401810BDE7
:10B84E00C20DD2B2FF2A01D0002A02D100220A6014
:10B85E0070477E3A0A60FF21C90588433F210906D9
:04B86E0040187047C7
:08B87200C1174840401A70475D
:10B87A0010B5002A0DD00446097848B200280AD427
:10B88A00002C00D02160002119605960411E8841B6
:0CB89A0010BD002010BD0120C04310BDF7
:10B8A600024601207F2901D9C043704711707047B5
:0CB8B600014661391A2900D22038704781
:0CB8C200014641391A2900D2203070479D
:0CB8CE00014661391A2900D22038704769
:0CB8DA00014641391A2900D22030704785
:10B8E60070B5012A09DB0C460546561C284621463A
:0CB8F600FFF7D4FE761E012EF8D870BDBE
:10B9020010B50C46436A01212046FFF767FF10BDC0
:10B91200010002000400060008000A000C001000EA
:08B9220020004000800000013C
:10B92A006E6F7420616C6C6F7765642C2070617225
:0FB93A00616D746572206C6F636B6564210A0028
:10B9490048414C5F434F4D50315F537461727420CD
:07B959004552524F520A0053
:10B9600048414C5F434F4D50325F537461727420B5
:07B970004552524F520A003C
:10B97700434F4E564552544552204552524F523A24
:10B9870020434F4E5645525445525F5354415254EB
:0BB997005550204552524F52210A002B
:10B9A200434F4E564552544552204552524F523AF9
:10B9B20020434F4E5645525445525F4552524F52C4
:10B9C2005F4F55545055545F564F4C545F544F4F30
:07B9D2005F484947480A00E5
:10B9D9004261747465726965206368617267656440
:10B9E90021204379636C65636F756E7465722B2BC7
:03B9F900210A0020
:10B9FC0048414C5F4144435F53746172745F444DE2
:07BA0C00413A204F4B0A00F4
:10BA13002D3E4D65737361676520746F2073686F86
:03BA23007274003A
:10BA26004A616E75617279004665627275617279F6
:10BA3600004D6172636800417072696C004D6179F6
:10BA4600004A756E65004A756C79004175677573B5
:10BA5600740053657074656D626572004F63746F30
:10BA6600626572004E6F76656D626572004465634D
:07BA7600656D6265720000BE
:07BA7D00414D00504D000097
:0FBA8400256120256220256520255420255900A5
:07BA9300286E756C6C2900A0
:10BA9A00443A5C70726F6A656B74655C6563735F68
:10BAAA00677265656E506F7765725061636B5C652E
:10BABA0063735F63656C6C4D6F6E5C6669726D77FC
:10BACA006172655C447269766572735C53544D3376
:10BADA0032473078785F48414C5F447269766572C4
:10BAEA005C5372635C73746D3332673078785F6865
:0ABAFA00616C5F636F6D702E6300D6
:10BB0400443A5C70726F6A656B74655C6563735FFD
:10BB1400677265656E506F7765725061636B5C65C3
:10BB240063735F63656C6C4D6F6E5C6669726D7791
:10BB34006172655C447269766572735C53544D330B
:10BB440032473078785F48414C5F44726976657259
:10BB54005C5372635C73746D3332673078785F68FA
:0EBB6400616C5F666C6173685F65782E6300CC
:10BB7200443A5C70726F6A656B74655C6563735F8F
:10BB8200677265656E506F7765725061636B5C6555
:10BB920063735F63656C6C4D6F6E5C6669726D7723
:10BBA2006172655C447269766572735C53544D339D
:10BBB20032473078785F48414C5F447269766572EB
:10BBC2005C5372635C73746D3332673078785F688C
:0ABBD200616C5F6770696F2E6300FD
:10BBDC00443A5C70726F6A656B74655C6563735F25
:10BBEC00677265656E506F7765725061636B5C65EB
:10BBFC0063735F63656C6C4D6F6E5C6669726D77B9
:10BC0C006172655C447269766572735C53544D3332
:10BC1C0032473078785F48414C5F44726976657280
:10BC2C005C5372635C73746D3332673078785F6821
:0ABC3C00616C5F756172742E630085
:10BC4600666163746F726520726573746F726520C6
:0ABC56002850696E292E2E2E0A00D8
:10BC60004558453A2053746F726520706172616D5A
:06BC7000657465720A0014
:10BC7600455845433A204170706C79204D4220501A
:0ABC86006172616D657465720A0059
:10BC9000455845433A20526573657420436F756E6D
:06BCA000746572730A00D6
:10BCA60048414C5F4441435F5374617274204F4B6B
:02BCB6000A0082
:10BCB80042414C414E4345525F496E6974204F4B97
:02BCC8000A0070
:10BCCA00434F4E564552544552204552524F523ACE
:10BCDA0020434F4E5645525445525F4552524F5299
:10BCEA005F4F55545055545F564F4C545F544F4F05
:06BCFA005F4C4F570A00E9
:10BD00004261747465726965206469736368617205
:06BD1000676564210A00D2
:10BD16004D696E75746520496E74657276616C6CDA
:0ABD260020636865636B73210A0057
:10BD30004E6577204D696E20566F6C746167652083
:0ABD400025642053617665640A0053
:10BD4A004E6577204D617820566F6C746167652067
:0ABD5A0025642053617665640A0039
:10BD640046697273742073746172742064657465B7
:06BD7400637465640A001F
:10BD7A00454550524F4D2046554C4C205245535440
:06BD8A004F5245210A00A2
:10BD9000454550524F4D2053544F524520434F4E2E
:06BDA000464947210A009C
:10BDA6004572726F72207768696C65207361766977
:10BDB6006E67206461746120746F20666C617368BD
:02BDC6000A0071
:0EBDC80075617274206572726F72200A0D0030
:02BDD600430028
:02BDD8002E003B
:10BDDA0053756E646179004D6F6E646179005475B4
:10BDEA006573646179005765646E6573646179008F
:10BDFA005468757273646179004672696461790086
:0ABE0A0053617475726461790000E1
:10BE1400443A5C70726F6A656B74655C6563735FEA
:10BE2400677265656E506F7765725061636B5C65B0
:10BE340063735F63656C6C4D6F6E5C6669726D777E
:10BE44006172655C447269766572735C53544D33F8
:10BE540032473078785F48414C5F44726976657246
:10BE64005C5372635C73746D3332673078785F68E7
:09BE7400616C5F6164632E6300E0
:10BE7D00443A5C70726F6A656B74655C6563735F81
:10BE8D00677265656E506F7765725061636B5C6547
:10BE9D0063735F63656C6C4D6F6E5C6669726D7715
:10BEAD006172655C447269766572735C53544D338F
:10BEBD0032473078785F48414C5F447269766572DD
:10BECD005C5372635C73746D3332673078785F687E
:09BEDD00616C5F6461632E630077
:10BEE600443A5C70726F6A656B74655C6563735F18
:10BEF600677265656E506F7765725061636B5C65DE
:10BF060063735F63656C6C4D6F6E5C6669726D77AB
:10BF16006172655C447269766572735C53544D3325
:10BF260032473078785F48414C5F44726976657273
:10BF36005C5372635C73746D3332673078785F6814
:09BF4600616C5F646D612E630003
:10BF4F00443A5C70726F6A656B74655C6563735FAE
:10BF5F00677265656E506F7765725061636B5C6574
:10BF6F0063735F63656C6C4D6F6E5C6669726D7742
:10BF7F006172655C447269766572735C53544D33BC
:10BF8F0032473078785F48414C5F4472697665720A
:10BF9F005C5372635C73746D3332673078785F68AB
:09BFAF00616C5F74696D2E630082
:10BFB800443A5C70726F6A656B74655C6563735F45
:10BFC800677265656E506F7765725061636B5C650B
:10BFD80063735F63656C6C4D6F6E5C6669726D77D9
:10BFE8006172655C447269766572735C53544D3353
:10BFF80032473078785F48414C5F447269766572A1
:10C008005C5372635C73746D3332673078785F6841
:0DC01800616C5F756172745F65782E630066
:10C0250066756C6C20726573746F72652E2E2E0AA0
:01C03500000A
:10C03600455845433A2053746F7265207769746892
:05C0460020736E0A00EA
:10C04B00455845433A2053617665206C6F636B20EE
:05C05B006B65790A008D
:10C06000554E4B4E4F574E20434F4D4D414E440A77
:01C0700000CF
:10C0710057726F6E6720706172616D65746572735E
:10C081002076616C75653A2066696C6520257320A0
:0DC091006F6E206C696E652025640D0A003D
:10C09E0048414C5F4441435F53657456616C75650E
:05C0AE00204F4B0A00C9
:10C0B30048414C5F4441435F53746172742045525D
:05C0C300524F520A007B
:10C0C80044432044432057616E646C6572206E6F50
:10C0D800742072756E6E696E672C20737461727449
:09C0E80020696D70756C730A008B
:10C0F10070726576696F757320636F6E666967200C
:09C1010070726573656E740A002A
:0DC10A0057726974696E6720534E210A0058
:10C117004572726F72207768696C652064656C651B
:10C1270074696E67206C6F67206461746120617247
:0DC13700656120696E20666C6173680A0006
:10C1440048414C5F41444345785F43616C69627286
:10C154006174696F6E5F53746172743A204F4B0A55
:01C1640000DA
:10C165004572726F722048414C5F4144435F53747E
:09C175006172745F444D410A003F
:10C17E002D3E4D657373616765207769746820770E
:09C18E00726F6E6720637263009A
:10C19700443A5C70726F6A656B74655C6563735F64
:10C1A700677265656E506F7765725061636B5C652A
:10C1B70063735F63656C6C4D6F6E5C6669726D77F8
:10C1C7006172655C7372635C6D6F646275732E6315
:01C1D7000067
:10C1D80053756E004D6F6E005475650057656400A9
:0DC1E80054687500467269005361740000D0
:10C1F5004A616E00466562004D61720041707200D1
:10C205004D6179004A756E004A756C00417567008D
:10C21500536570004F6374004E6F7600446563008C
:01C225000018
:01C226000017
:09C22700256D2F25642F257900F7
:09C2300025483A254D3A2553003A
:0DC239000007032004170201085710408081
:05C246002D494E4600E9
:05C24B002D696E660084
:05C250002B494E4600E1
:05C255002B696E66007C
:02C25A00FFFFE4
:04C25C008531000820
:10C26000443A5C70726F6A656B74655C6563735F9A
:10C27000677265656E506F7765725061636B5C6560
:10C2800063735F63656C6C4D6F6E5C6669726D772E
:10C290006172655C447269766572735C53544D33A8
:10C2A00032473078785F48414C5F447269766572F6
:10C2B0005C5372635C73746D3332673078785F6897
:0CC2C000616C5F6164635F65782E630051
:10C2CC00443A5C70726F6A656B74655C6563735F2E
:10C2DC00677265656E506F7765725061636B5C65F4
:10C2EC0063735F63656C6C4D6F6E5C6669726D77C2
:10C2FC006172655C447269766572735C53544D333C
:10C30C0032473078785F48414C5F44726976657289
:10C31C005C5372635C73746D3332673078785F682A
:0CC32C00616C5F74696D5F65782E6300C2
:08C338000101010307010000EF
:08C340000804020408010101D8
:10C348007265616420636F6E6669672E2E2E0A001F
:10C35800455845433A205265736574204D696E20EF
:10C36800616E64204D61782056616C7565730A00B2
:10C3780048414C5F434F4D50315F53746172742094
:04C388004F4B0A000D
:10C38C0048414C5F434F4D50325F5374617274207F
:04C39C004F4B0A00F9
:10C3A0004E6577204D696E2054656D702E20256492
:08C3B0002053617665640A0068
:10C3B8004E6577204D61782054656D702E20256478
:08C3C8002053617665640A0050
:10C3D000486F757220496E74657276616C6C20636B
:08C3E0006865636B73210A001C
:10C3E800454550524F4D2053544F5245204C4F47CE
:08C3F8002044415441210A00D8
:10C4000048414C5F41444345785F43616C696272C7
:10C410006174696F6E5F53746172743A2045525251
:04C420004F520A006D
:10C424004572726F722C2072656164206F6E6C7934
:0CC43400205265676973746572210A006C
:10C4400050726F74656374656420526567697374B4
:10C4500065722C207772697465206E6F7420616C30
:08C460006C6F776564210A008E
:10C46800202020202020202020682828282820205C
:10C4780020202020202020202020202020202020B4
:10C48800481010101010101010101010101010106C
:10C49800848484848484848484841010101010100C
:10C4A8001081818181818101010101010101010165
:10C4B8000101010101010101010101101010101019
:10C4C8001082828282828202020202020202020236
:10C4D80002020202020202020202021010101020DE
:10C4E80030313233343536373839414243444546A2
:10C4F80030313233343536373839616263646566D2
:04C508004E414E0052
:04C50C006E616E00EE
:10C5100000B506480649884205D00268043003B4D5
:10C52000904703BCF7E708BC184700005CC200084E
:04C5300060C20008DD
:10C534009DC5000800000020480B0000AFC500089E
:10C54400480B002058C500083DB3000811C5000879
:04C554006B3100083F
:10C5580018A0B20008A0B20008A0B20008A0B2005B
:10C5680008A0B200080024F4000AFE000F340B00F3
:10C5780020380B00203C0B002000000202FD00FDCB
:10C5880002010101FB00E70204010000010298001A
:04C59800800000001F
:10C59C00206861680834002200E042540139FCD55F
:02C5AC007047D6
:10C5AE002068616808340A780131802A11D009D3D5
:10C5BE000B7801315242FF32013203700130013AE1
:10C5CE00FBD5F0E70B78037001300131013AF9D554
:04C5DE00E9E77047D2
:10C5E200FFFFFFFFFFFFFFFFFFFFFFFFFFFFFFFF59
:10C5F200FFFFFFFFFFFFFFFFFFFFFFFFFFFFFFFF49
:10C60200FFFFFFFFFFFFFFFFFFFFFFFFFFFFFFFF38
:10C61200FFFFFFFFFFFFFFFFFFFFFFFFFFFFFFFF28
:020000040801F1
:04EFFC00642CCCC7EE
:040000050800B777C1
:00000001FF
